:020000040000FA
:100000003039012055030000790300007B03000014
:100010007D0300007F0300008103000083030000D4
:1000200083030000830300008303000083030000B8
:100030008303000083030000EF0200000D34000082
:10004000E9060000F3060000FD06000007070000B7
:1000500011070000090A0000130A00002D09000022
:1000600033080000A1080000AB080000B50800003C
:10007000BF080000D3080000450600004F0600003E
:100080005906000063060000770A000069090000B5
:10009000730900007D090000870900009109000034
:1000A0009B09000027060000310600003B06000007
:1000B00055090000D50600001B07000025070000B9
:1000C0002F0700001D0A000037090000A5090000E5
:1000D000AF0900003D0800009F060000A9060000CF
:1000E000CB060000290800006D0A0000C9080000C6
:1000F000630A0000590A00006D0600007706000040
:10010000810600008B060000C106000039070000D0
:10011000430700004D070000410900004B090000A3
:10012000270A0000310A00003B0A0000450A0000CF
:100130004F0A00004708000051080000B9090000FC
:10014000C3090000CD090000D7090000DF06000048
:10015000050900000F0900005B08000065080000A9
:100160005707000061070000190900005F0900003F
:100170006B070000750700007F070000890700007B
:10018000930700009D070000A7070000B1070000CB
:10019000BB070000C5070000CF070000D90700001B
:1001A000E3070000ED070000F7070000010800006A
:1001B0000B08000015080000230900009506000048
:1001C000B306000097080000E1090000EB090000F9
:1001D000F5090000FF0900006F0800007908000021
:1001E000DD0800001D060000E7080000F10800001F
:1001F000FB080000830800008D0800001F080000B5
:10020000DFF80CD000F028F9004800472D58000016
:1002100030390120EFF3108072B67047EFF3108091
:100220007047EFF3108062B6704730BF704780F3BD
:1002300011887047EFF31180704700000138FDD13D
:100240007047000072B6704762B67047EFF31080D7
:1002500072B6704780F31088704730BF704720BF78
:100260007047B0FA80F0704790FAA0F0B0FA80F0D2
:10027000704790FAA0F07047EFF3098141B1F1EEB9
:10028000101A40F8041D20ED200A29490A68106060
:100290007047B0EC200A02C8E1EE101A25490A683E
:1002A00010607047EFF3108072B6704780F31088CB
:1002B000704721484FF0FF010170002080F309884A
:1002C0001E48016881F308881D48012101701D48FE
:1002D0004FF08051016062B6FEE71A484FF080513E
:1002E0000160704717484FF080510160704772B647
:1002F000EFF3098028B1203880E8F00F0C49096835
:10030000086000B5104880475DF804EB0F481049BD
:100310000A780270064807490A680260106890E887
:10032000F00F203080F309884EF0F40E62B670476B
:10033000340000203C00002022ED00E06C00002092
:100340002E00002004ED00E0792F000023000020A3
:1003500024000020DFF83000016841F470010160E2
:10036000BFF34F8FDFF82400016821F040410160A6
:10037000BFF36F8F06480047FEE7FEE7FEE7FEE7A4
:10038000FEE7FEE7FEE7000088ED00E034EF00E066
:100390000102000040EA01039B0703D009E008C9FD
:1003A000121F08C0042AFAD203E011F8013B00F83A
:1003B000013B521EF9D27047D2B201E000F8012B86
:1003C000491EFBD270470022F6E710B513460A46D5
:1003D00004461946FFF7F0FF204610BD421E12F8F2
:1003E000013F002BFBD111F8013B02F8013B002B30
:1003F000F9D1704710B5002200E0521C835C8C5C80
:10040000A34201D1002BF8D1D8B2E1B2401A10BDFD
:1004100030B504460020034600E05B1C934203D243
:10042000E05CCD5C401BF8D030BD30B50B460146DA
:1004300000202022012409E021FA02F59D4205D383
:1004400003FA02F5491B04FA02F52844151EA2F12D
:100450000102F1DC30BD0000064C074D06E0E0680B
:1004600040F0010394E8070098471034AC42F6D3FB
:10047000FFF7CAFE10AC000030AC000070B58C185D
:1004800010F8015B15F0070301D110F8013B2A11A8
:1004900006D110F8012B03E010F8016B01F8016B95
:1004A0005B1EF9D12B0705D40023521E0DD401F891
:1004B000013BFAE710F8013BCB1A921C03E013F85A
:1004C000015B01F8015B521EF9D5A142D8D300208F
:1004D00070BD000000B585B0032000214FF480728C
:1004E0000E4BCDE90132CDE90310062003460C4A3C
:1004F00000900C4802F036FA032000214FF480727D
:10050000094BCDE90132CDE9031007200346074A24
:100510000090074802F026FA05B000BD2C2F0120FC
:1005200028330120D93C00002C330120283701203A
:10053000DD3F000086B000F041F800F0C9FA044643
:100540004FF47A70B4FBF0F5284602F073FF00F028
:100550007CFE02F0DBF901F007FD204600F096FC7E
:1005600000F09AFC09F0E4FF0C4803C8CDE9000153
:100570000B48006805900B48006804900A48006822
:100580000390DDE9041203F055FDFFF7A3FF03E03C
:100590004FF47A7002F0F4FCFAE70000C00100208A
:1005A000B8010020B4010020B0010020704770475E
:1005B00070477047704770477047704710B500F03C
:1005C0005FFA00F0D9FA10BD10B50446702C04D2C1
:1005D00004F11001C8B200F03FFE10BD70B5044632
:1005E000002600BF00BFFFF731FE064600BF00BF78
:1005F00001F024FE00BF00BF3046FFF72BFE00BF16
:1006000000BF702C04D2044850F8245005B1A8470C
:1006100001F02EFE70BD00002806002010B56920F4
:10062000FFF7DCFF10BD10B51920FFF7D7FF10BD95
:1006300010B51A20FFF7D2FF10BD10B51B20FFF731
:10064000CDFF10BD10B50E20FFF7C8FF10BD10B5CF
:100650000F20FFF7C3FF10BD10B51020FFF7BEFF3E
:1006600010BD10B51120FFF7B9FF10BD10B52E2039
:10067000FFF7B4FF10BD10B52F20FFF7AFFF10BD7F
:1006800010B53020FFF7AAFF10BD10B53120FFF7DD
:10069000A5FF10BD10B55F20FFF7A0FF10BD10B57E
:1006A0002620FFF79BFF10BD10B52720FFF796FF10
:1006B00010BD10B56020FFF791FF10BD00BFFEE731
:1006C00010B53220FFF78AFF10BD10B52820FFF7C4
:1006D00085FF10BD10B51D20FFF780FF10BD10B5C0
:1006E0004320FFF77BFF10BD10B50020FFF776FF1A
:1006F00010BD10B50120FFF771FF10BD10B502202D
:10070000FFF76CFF10BD10B50320FFF767FF10BDAA
:1007100010B50420FFF762FF10BD10B51E20FFF7D3
:100720005DFF10BD10B51F20FFF758FF10BD10B5BD
:100730002020FFF753FF10BD10B53320FFF74EFF09
:1007400010BD10B53420FFF749FF10BD10B535209E
:10075000FFF744FF10BD10B54820FFF73FFF10BD65
:1007600010B54920FFF73AFF10BD10B54C20FFF738
:1007700035FF10BD10B54D20FFF730FF10BD10B58F
:100780004E20FFF72BFF10BD10B54F20FFF726FFBF
:1007900010BD10B55020FFF721FF10BD10B551203E
:1007A000FFF71CFF10BD10B55220FFF717FF10BD5B
:1007B00010B55320FFF712FF10BD10B55420FFF7FE
:1007C0000DFF10BD10B55520FFF708FF10BD10B587
:1007D0005620FFF703FF10BD10B55720FFF7FEFEB0
:1007E00010BD10B55820FFF7F9FE10BD10B5592007
:1007F000FFF7F4FE10BD10B55A20FFF7EFFE10BD55
:1008000010B55B20FFF7EAFE10BD10B55C20FFF7C6
:10081000E5FE10BD10B55D20FFF7E0FE10BD10B580
:100820006F20FFF7DBFE10BD10B52920FFF7D6FEC5
:1008300010BD10B50820FFF7D1FE10BD10B5252062
:10084000FFF7CCFE10BD10B53D20FFF7C7FE10BD71
:1008500010B53E20FFF7C2FE10BD10B54620FFF7D1
:10086000BDFE10BD10B54720FFF7B8FE10BD10B596
:100870006620FFF7B3FE10BD10B56720FFF7AEFE90
:1008800010BD10B56D20FFF7A9FE10BD10B56E208C
:10089000FFF7A4FE10BD10B56120FFF79FFE10BD4D
:1008A00010B50920FFF79AFE10BD10B50A20FFF71A
:1008B00095FE10BD10B50B20FFF790FE10BD10B5D2
:1008C0000C20FFF78BFE10BD10B52B20FFF786FE26
:1008D00010BD10B50D20FFF781FE10BD10B56820CA
:1008E000FFF77CFE10BD10B56A20FFF777FE10BD44
:1008F00010B56B20FFF772FE10BD10B56C20FFF72E
:100900006DFE10BD10B54420FFF768FE10BD10B598
:100910004520FFF763FE10BD10B54A20FFF75EFECD
:1009200010BD10B55E20FFF759FE10BD10B50720B1
:10093000FFF754FE10BD10B52220FFF74FFE10BD8B
:1009400010B53620FFF74AFE10BD10B53720FFF76F
:1009500045FE10BD10B51C20FFF740FE10BD10B5C0
:100960004B20FFF73BFE10BD10B51320FFF736FEFE
:1009700010BD10B51420FFF731FE10BD10B51520C5
:10098000FFF72CFE10BD10B51620FFF727FE10BD97
:1009900010B51720FFF722FE10BD10B51820FFF785
:1009A0001DFE10BD10B52320FFF718FE10BD10B5B9
:1009B0002420FFF713FE10BD10B53F20FFF70EFEF9
:1009C00010BD10B54020FFF709FE10BD10B5412045
:1009D000FFF704FE10BD10B54220FFF7FFFD10BD6C
:1009E00010B56220FFF7FAFD10BD10B56320FFF7C8
:1009F000F5FD10BD10B56420FFF7F0FD10BD10B57A
:100A00006520FFF7EBFD10BD10B50520FFF7E6FDF3
:100A100010BD10B50620FFF7E1FD10BD10B5212077
:100A2000FFF7DCFD10BD10B53820FFF7D7FD10BD76
:100A300010B53920FFF7D2FD10BD10B53A20FFF7F1
:100A4000CDFD10BD10B53B20FFF7C8FD10BD10B5A2
:100A50003C20FFF7C3FD10BD10B52D20FFF7BEFDF4
:100A600010BD10B52C20FFF7B9FD10BD10B52A2020
:100A7000FFF7B4FD10BD10B51220FFF7AFFD10BD9C
:100A800010B5002404E0E0B2034900F007F8641C4C
:100A9000702CF8D310BD0000BD06000070B50446F0
:100AA0000D460026702C10D200BF00BFFFF7CEFB12
:100AB000064600BF00BF054840F8245000BF00BFF5
:100AC0003046FFF7C7FB00BF00BF70BD28060020FF
:100AD0002DE9F043DFF894C0DCF8B0C0CCF3007C23
:100AE000BCF1000F3ED0DFF884C0DCF860C1CCF36D
:100AF0008A24DFF878C0DCF860C1CCF30A0303EB8A
:100B00009422DFF868C0DCF864C1CCF30425DFF878
:100B10005CC0DCF864C10CF01F06DFF850C0DCF8E4
:100B2000B0C0CCF3036111B1032904D101E0104935
:100B300002E0104900E000BF00BF01FB02F805F130
:100B4000010C06F101090CFB09FCB8FBFCF0DFF815
:100B50001CC0DCF8B0C0CCF3090C0CF10107B0FBF1
:100B6000F7F000E00020BDE8F083000000E00F4057
:100B70000024F40040787D012948C06F20F01C005B
:100B80002749C8670846C06F40F01000C86724486E
:100B9000C0300068234908402149C1F8C0002048FE
:100BA000C0300068204908431D49C031086048062C
:100BB0001B49B03108604FF04C70086060201B4941
:100BC000086004201649C1F864011848A03800687C
:100BD000144908401249C1F8C0001448A038006800
:100BE000134908430E49C1F8C0000846D0F8600117
:100BF00040F40000C1F8600100BF0C4808300068F4
:100C000000F0010080F001000028F6D10448B03067
:100C10000068084908430249C1F8B0007047000065
:100C200000E00F4010FC10FC8100010060E10F406B
:100C300085018501030000900148006870470000AD
:100C4000540100202DE9F04104460F4615461E468A
:100C50008DB9204603F034FC24B93946114804F01C
:100C600019FE05E0012C03D139460F4804F012FEAD
:100C70000020BDE8F081012D10D1204603F020FCBA
:100C800024B93146074805F055FE05E0012C03D193
:100C90003146054805F04EFE0020EAE74FF0FF30F0
:100CA000E7E7000000000240001002402DE9F04795
:100CB0000646894617461D464FF0000AFFF7F2FA2E
:100CC000824635B95046FFF7F1FA4FF0FF30BDE8E4
:100CD000F08716B9DFF8E8800AE0012E02D1DFF8CC
:100CE000E48005E05046FFF7E1FA4FF0FF30EEE711
:100CF00000BF404600F0C4FF0028FAD10122494657
:100D0000404601F00FF8012D1BD10721404600F0AD
:100D1000C0FF404600F0C9FF20B15046FFF7C6FAB9
:100D2000A81ED4E700BF404600F0AAFF0028FAD171
:100D3000404600F0B0FF38705046FFF7B7FA002089
:100D4000C5E7002434E024B90B21404600F0A1FFA0
:100D50000BE0681EA04204D10521404600F099FF37
:100D600003E00921404600F094FF404600F09DFF5B
:100D700098B1681EA0420AD0404600F096FF00F0ED
:100D80001000102803D00421404600F082FF504696
:100D9000FFF78CFA4FF0FF3099E700BF404600F0B4
:100DA0006FFF0028FAD1404600F075FF3855641CEB
:100DB000AC42C8D35046FFF779FA002087E700001D
:100DC00000000240001002402DE9F0470646884628
:100DD00017461D464FF0000AFFF764FA824615B128
:100DE00046B1012E06D05046FFF760FA4FF0FF30B3
:100DF000BDE8F0870EB9234800E02348814600BFD4
:100E0000484600F03DFF0028FAD1002241464846FE
:100E100000F088FF00242DE0395D484600F03EFFD9
:100E200024B90321484600F034FF0BE0681EA042BD
:100E300004D10521484600F02CFF03E0012148467B
:100E400000F027FF484600F030FF60B1681EA04266
:100E500003D00421484600F01CFF5046FFF726FA55
:100E60004FF0FF30C4E700BF484600F009FF0028FC
:100E7000FAD1641CAC42CFD35046FFF717FA0020DA
:100E8000B6E700000000024000100240014908607F
:100E900070470000540100207047000010B54FF467
:100EA0008073034A0349044800F0A6F910BD00000E
:100EB00058010020F022012000C0004010B54FF47E
:100EC0008073034A0349044800F096F910BD0000FE
:100ED00060010020F023012000D0004010B54FF445
:100EE0008073034A0349044800F086F910BD0000EE
:100EF00068010020F024012000E0004010B54FF40C
:100F00008073034A0349044800F076F910BD0000DD
:100F100070010020F025012000F0004010B54FF4D2
:100F20008073034A0349044800F066F910BD0000CD
:100F300078010020F02601200000014010B54FF498
:100F40008073034A0349044800F056F910BD0000BD
:100F500080010020F02701200010014010B54FF45F
:100F60008073034A0349044800F046F910BD0000AD
:100F700088010020F02801200020014010B54FF426
:100F80008073034A0349044800F036F910BD00009D
:100F900090010020F0290120003001402DE9F041AE
:100FA0008CB080460C4615461E46129FB8F1080FBD
:100FB00077D2DFE808F004203C597794AFCA1520B7
:100FC000714905220223CDE90967CDE90745CDE93D
:100FD0000332CDE90510012040F20141CDE90001C5
:100FE0004FF04023694A6A4902906A4802F0B6FF0E
:100FF0000CB0BDE8F0811620674906220223CDE936
:101000000967CDE90745CDE90332CDE90510012097
:1010100062494FF00112624BCDE900210290614A12
:101020005B49491C5B48401C02F098FFE0E7312017
:101030005D4921228023CDE90967CDE90745CDE946
:101040000332CDE90510402041F6014141F601028D
:101050004FF04023CDE900210290544A4C494D48BD
:10106000801C02F07BFFC3E748205149382220232F
:10107000CDE90967CDE90745CDE90332CDE9051092
:10108000102041F2014141F201024FF04023CDE92D
:1010900000210290474A3E493E48C01C02F05EFFD4
:1010A000A6E76DE04920444939220823CDE90967C4
:1010B000CDE90745CDE90332CDE90510042040F61E
:1010C000014140F601024FF04023CDE9002102909A
:1010D0003A4A2F492F48001D02F040FF88E74A2076
:1010E00037493A228023CDE90967CDE90745CDE9A3
:1010F0000332CDE9051040203249334A334BCDE964
:1011000000210290324A2249891C2248401D02F0E7
:1011100025FF6DE74B202F493B220223CDE90967CC
:10112000CDE90745CDE90332CDE9051001202A4973
:101130002A4A2B4BCDE9002102902A4A14490D314D
:101140001448801D02F00AFF52E74C2026493C2239
:101150002023CDE90967CDE90745CDE90332CDE983
:10116000051010202149224A184BCDE90021029098
:10117000204A0749891C0748C01D02F0EFFE37E7E7
:101180004FF0FF3034E700009D0E000000C000402B
:10119000000800F0001800F0BD0E0000010401007E
:1011A0000050004000D00040DD0E000000E0004094
:1011B000FD0E000000F000401D0F00000000014087
:1011C0003D0F0000011C02000118020000600040F9
:1011D000001001405D0F000001040D0001000D0032
:1011E00000500640002001407D0F00000114020065
:1011F00001100200003001402DE9F04107460D4684
:1012000014461E460121384602F0A2FE80464146A1
:10121000384602F097FE01F011F80DE0384602F072
:1012200039FE216868542068401C20602068B0FBAB
:10123000F6F106FB11002060384602F03DFE002862
:10124000ECD101F015F8BDE8F08110B500F0FAF826
:1012500000F0C0F810BD00002DE9F04104464FF049
:101260000008102C6BD2DFE804F0080E0F101429D0
:101270003E090A0B0C11120D135300BF00BF00BF33
:1012800000BF00BF89E000BF00BF00BF00BF00BFBC
:1012900083E000BF00BFFEF7D9FF804600BF00BF5C
:1012A0003F48006840F480303D49086000BF00BFFF
:1012B0004046FEF7CFFF00BF00BF6EE000BF00BF9B
:1012C000FEF7C4FF804600BF00BF3548006840F409
:1012D00000303349086000BF00BF4046FEF7BAFF48
:1012E00000BF00BF59E000BF00BFFEF7AFFF804660
:1012F00000BF00BF2A48006840F4802028490860E9
:1013000000BF00BF4046FEF7A5FF00BF00BF44E09E
:1013100000BF00BFFEF79AFF804600BF00BF4FF03E
:10132000E020006940F001004FF0E021086100BFBB
:1013300000BF4046FEF78EFF00BF00BF2DE04FF01C
:10134000E0204068401C102101EB4010C7B2BC42B5
:1013500022DAA4F11000C11700EBD161C1F34715E7
:10136000C11700EBD1614911A0EB4111CEB200BF12
:1013700000BFFEF76BFF804600BF00BF0120B040FA
:10138000A90001F1E021C1F8000100BF00BF404603
:10139000FEF760FF00BF00BF00BF00BFBDE8F081E7
:1013A00024ED00E010B5002400BF00BFFEF74EFFA3
:1013B000044600BF00BF1021054800F0CBFD00BF70
:1013C00000BF2046FEF746FF00BF00BF10BD000073
:1013D000D001002010B5FFF7E5FF10BD2DE9F04169
:1013E00005460C46002714B900BF00F029F81DB9C6
:1013F0000A202080BDE8F0811021284602F0B1FCCF
:101400000646102E15D200BF00BFFEF71FFF07468D
:1014100000BF00BF10222946084802F07FFC00BF31
:1014200000BF3846FEF716FF00BF00BF0020208037
:1014300002E04FF47A70208000BFDBE7D00100208B
:1014400000BFFEE710B500200249086000F00AF86E
:1014500010BD000000000020014908607047000036
:101460000000002010B50A48006840F0807008496C
:1014700008600020074948600846006840F0010005
:101480000860FFF725FB04462046FFF7E5FF10BD87
:10149000FCED00E0001000E00146002902DA4FF008
:1014A000FF3070470020FCE770B50446601C00F078
:1014B000B9F80546FFF7F0FF002802DA4FF0FF30D9
:1014C00070BDA01C00F09EF80546FFF7E5FF002860
:1014D00002DA4FF0FF30F3E7E01C00F08BF805462E
:1014E000FFF7DAFF002802DA4FF0FF30E8E7201DAF
:1014F00000F078F80546FFF7CFFF002802DA4FF03A
:10150000FF30DDE7601D00F085F80546FFF7C4FFFA
:10151000002802DA4FF0FF30D2E7A01D00F08AF871
:101520000546FFF7B9FF002802DA4FF0FF30C7E7A2
:101530000020C5E770B504460D461448047000232A
:101540001A4629460078FFF77DFB06463046FFF72E
:10155000A3FF002802DA4FF0FF3070BD00F072F8F0
:1015600006463046FFF798FF002802DA4FF0FF30BA
:10157000F3E700F00DF806463046FFF78DFF002830
:1015800002DA4FF0FF30E8E70020E6E7AC01002088
:1015900010B55E21202002F0ADFB0446FFF77CFF72
:1015A000002802DA4FF0FF3010BDC721212002F0E1
:1015B000A1FB0446FFF770FF002802DA4FF0FF306E
:1015C000F2E70121222002F095FB0446FFF764FFB9
:1015D000002802DA4FF0FF30E6E74021072002F052
:1015E00089FBE1E710B5044630222146042002F0D1
:1015F0003BFB10BD10B5044630222146022002F00C
:1016000033FB10BD10B5044670222146012002F0C4
:101610002BFB10BD10B5044610222146052002F018
:1016200023FB10BD10B5044670222146002002F0B5
:101630001BFB10BD10B50446F0222146062002F027
:1016400013FB10BD10B52021082002F053FB044607
:10165000FFF722FF002802DA4FF0FF3010BD4521CE
:10166000092002F047FBF9E738B504460D46002093
:1016700003466022294600902046FFF78FFC38BDC4
:1016800010B50346CC00443418591070040A547045
:10169000040C9470040ED470CC00403418591071AE
:1016A000040A547110BD10B5CB004033C3586FF31A
:1016B0000F0314792343547943EA0424CB004033C5
:1016C000C4501378547843EA0423947843EA0443DB
:1016D000D47843EA0464CB004433C45010BD000006
:1016E00070B5D0F8185C156005680C4E35400D607B
:1016F000D0F8DC4004F480351DB1C4F30D051D6045
:101700000AE0056805F480151DB14FF420551D60F1
:1017100002E04FF400651D6070BD0000FF7E5F7A3F
:1017200030B504680A4D2C400C4344F40044046076
:1017300023B143F48034C0F8DC4005E0D0F8DC404D
:1017400024F48034C0F8DC40C0F8182C30BD000010
:101750000C81A0854268024B1A400A4342607047E0
:1017600000F8FE7FF0B50446DDE9055700BFDFF85D
:1017700094C0DCF800C00CF0010CBCF1000FF6D1F5
:1017800042EA870C4CF08000202D01D8202B03D991
:1017900040F08070ED08DB08AB4202D140EA052042
:1017A00007E04FF4000C4CEA052C4CEA434C4CEAA1
:1017B0000000C4F8000CDFF850C0DCF81460002012
:1017C0000DE0DFF844C05CF830C08C4506D3DFF88C
:1017D00038C00CEBC00CDCF8046002E0401C0328AD
:1017E000EFD300BFD4F810C02CF03C0C4CEA060C30
:1017F000C4F810C04FF0FF3CC4F80CC1C4F810C1CD
:10180000F0BD000000CC0E404CA5000044F24502A3
:101810000A400AB141F4803142F2BA720A400AB178
:1018200041F4004121F000421AB121F00042C0F819
:10183000142C01F000422AB1D0F8D82F42F0010256
:10184000C0F8D82F704744F245020A400AB141F46B
:10185000803142F2BA720A400AB141F4004121F0EB
:10186000004232B1D0F81C2C21F000431A43C0F8DA
:101870001C2C01F000422AB1D0F8D42F42F0010212
:10188000C0F8D42F7047000010B50246D2F8140CEF
:10189000094C204021B1D2F81C4C44F0F0442040C7
:1018A00011B1D2F8D83F01E0D2F8D03F03F00104E3
:1018B0000CB140F0004010BDFFFF01FC70B50546C3
:1018C0000C46C5F8C44F04F0404060B9134802F01C
:1018D000A9FA00BF114802F089FA0028FAD042F2B2
:1018E0001070FEF7ABFC04F04040B0F1404F06D161
:1018F0000B48006840F480300949086005E008485A
:10190000006820F4803006490860064800F042F87C
:101910004FF47A70FEF792FC70BD0000003000F0CA
:10192000C8CF0E4000C00E40034600BF186900F04B
:1019300001000028FAD1186900F03C0040EA82104A
:1019400040EAC120401C186100BF186900F0010086
:101950000028FAD1586980B2704710B500BF0469F9
:1019600004F00104002CFAD14361046904F03C0442
:1019700044EA821444EAC124E41C046100BF0469FF
:1019800004F00104002CFAD110BD0146C86A00F031
:1019900061007047D0F8001C41F00101C0F8001C44
:1019A00000BFD0F8001C01F001010029F9D17047F7
:1019B000C0F80C1C7047D0F8181C41F00201C0F8A8
:1019C000181C016841F00401016070470146D1F81C
:1019D00028077047C0F8101C70470021C0F8041C8D
:1019E0007047D0F8181C41F40051C0F8181C016869
:1019F00041F008010160704702F001031BB1D0F80B
:101A000000340B4302E0D0F800348B43C0F80034BC
:101A100002F002031BB1D0F820340B4302E0D0F8EF
:101A200020348B43C0F8203470470000F0B55F4D80
:101A30002D685F4E35405F4EB5421AD0002416E047
:101A40000125A5400D4085B1D0F8C45F670003268D
:101A5000BE40B543C0F8C45FD0F8C45F6700C2F3AE
:101A60004116BE403543C0F8C45F651CECB2082C7B
:101A7000E6DB02F001051DB1D0F800550D4302E090
:101A8000D0F800558D43C0F8005502F002051DB195
:101A9000D0F804550D4302E0D0F804558D43C0F84A
:101AA000045502F004051DB1D0F808550D4302E0BD
:101AB000D0F808558D43C0F8085502F008051DB14F
:101AC000D0F818550D4302E0D0F818558D43C0F8F2
:101AD0001855364D2D68364E3540364EB5420BD032
:101AE00002F010051DB1D0F83C550D4302E0D0F8CE
:101AF0003C558D43C0F83C5503F001051DB1D0F8AD
:101B00000C550D4302E0D0F80C558D43C0F80C5530
:101B100003F002051DB1D0F810550D4302E0D0F8D6
:101B200010558D43C0F8105503F004051DB1D0F8D1
:101B300014550D4302E0D0F814558D43C0F81455E8
:101B400003F008051DB1D0F81C550D4302E0D0F894
:101B50001C558D43C0F81C55144D2D68144E35404E
:101B6000144EB54217D003F400751DB1D0F844559A
:101B70000D4302E0D0F844558D43C0F8445503F4BA
:101B800040751DB1D0F840550D4302E0D0F84055E6
:101B90008D43C0F840551BB9D0F828550D4302E0DD
:101BA000D0F828558D43C0F82855F0BD00E00F400F
:101BB0000000FF700000051010B50146C1F307409A
:101BC0000F4BDB6E01248440234033B1012303EB30
:101BD00040030C4C54F8230003E04300094C54F834
:101BE0002300C1F30722D0F82C350F249440A343DF
:101BF00001F00F0494402343C0F82C3510BD0000C1
:101C000000E00F40FCA6000030B504460D4602225D
:101C100029462046FFF7F0FE082366222946204683
:101C2000FFF704FF30BD30B504460D4602222946B9
:101C30002046FFF7E1FE0923012229462046FFF74F
:101C4000F5FE30BD30B504460D4602222946204639
:101C5000FFF7D2FE0823012229462046FFF7E6FEC1
:101C600030BD30B504460D46022229462046FFF716
:101C7000C3FE0823012229462046FFF7D7FE30BDC8
:101C80000146486800F0010008B1012070470020BB
:101C9000FCE7416070470146886870478160704783
:101CA000016A41F01001016270470246516801F07B
:101CB000010008B10020704701F0120010B101F0DE
:101CC0001C00F8E70020F6E770B503460C46164600
:101CD0001846FFF7E5FF012E01D10F4A00E00F4A39
:101CE000142000FB0240401E02EB82018900B0FB81
:101CF000F1F0451EDD60D3F8C00F00F0010048B1DF
:101D000007482044401E0649B0FBF1F0451E45F04F
:101D10008000D86070BD0000801A0600A086010017
:101D20008047370142EA410303607047016A41F08E
:101D3000200101620121C0F80418704700B5024675
:101D40000B461046FFF7F2FFC2F8003800BD000056
:101D500010B5002426E0002004EBC4014A4A02EB3F
:101D60008101086204EBC40102EB8101486004EBCD
:101D7000C40102EB81018860172C01D1104605E0F7
:101D8000601C00EBC000404901EB800004EBC40183
:101D90003D4A02EB8101C8603C4804EBC40142F8B3
:101DA0002100641C182CD6D3002039498860C860F3
:101DB000002459E0032240F2EC51104604F06AFA84
:101DC00004EBC401334A02EB810108624FF4804006
:101DD00004EBC40102EB8101486004EBC40011462E
:101DE00001EB8000006A18B304EBC40001EB800033
:101DF000006A406804EBC40102EB8101886004EBD7
:101E0000C400114601EB8000406804EBC40102EB02
:101E10008101096A4989084304EBC40102EB81018D
:101E200048604FF0004004EBC40142F821000AE092
:101E3000002004EBC401174A02EB8101886004EB27
:101E4000C40142F82100072C01D1124805E0601CB2
:101E500000EBC0000F4901EB800004EBC4010D4A08
:101E600002EB8101C860641C082CA3D30020084940
:101E70008860C86007490848FFF79AFD024906488C
:101E8000FFF7A8FD10BD0000701E01200000D0402B
:101E900018010020D021012000C00E40042806D1E6
:101EA0001949096841F48031174A11602BE005286F
:101EB00006D11549096841F40031134A116022E046
:101EC000062806D11049096841F480210E4A1160A4
:101ED00019E00F2808D14FF0E021096941F0020113
:101EE0004FF0E02211610EE010280CD3A0F1100198
:101EF00001F01F0201219140A0F110025209034B91
:101F000053F822201160704724ED00E048A800003B
:101F100010B5FEF786F908B1012010BD0020FCE7DE
:101F200010B50A4683080A4C54F823301968830711
:101F3000DC0EFF23A34099438307DB0E02FA03F371
:101F400019438308024C54F82330196010BD000077
:101F5000ACA7000030B505460C46224600212846B5
:101F600000F026F830BD00000D480E490160014622
:101F7000416000218160C160016141618161C16195
:101F800001620163C162416207498163C1634FF429
:101F90008061016441640146044A11607047000099
:101FA000E0010020484541502802002004000020A4
:101FB0002DE9F04103460C4617460FB9BDE8F08104
:101FC00003B9FBE70025002202E02D022543521C45
:101FD000042AFAD3384603F0030C1946BCF1000F6B
:101FE00008D0624603E001F8014B401E521C08B1C4
:101FF000042AF8D30E4601E020C6001F0428FBD2B5
:10200000314602E001F8014B401E0028FAD100BF22
:10201000D4E700001D481E481E481F481F4820489E
:102020002048214821482248224823482348244860
:102030002448254825482648264827482748284830
:102040002848294829482A482A482B482B482C4800
:102050002C482D482D482E482E482F482F483048D0
:1020600030483148314832483248334833483448A0
:102070003448354835483648364837483748384870
:1020800038483948394800BF7047000098A9000017
:102090009CA90000A2A90000A4A90000A0A900001A
:1020A000A6A90000A8A90000AAA90000ACA90000E8
:1020B000AEA90000B0A90000B2A90000B4A90000B8
:1020C000B6A90000B8A90000BAA90000BCA9000088
:1020D000BEA90000C0A90000C2A90000C4A9000058
:1020E000C6A90000C8A90000CAA90000CCA9000028
:1020F000CEA90000D0A90000D2A90000D4A90000F8
:10210000D6A90000D8A90000DAA90000DCA90000C7
:10211000DEA90000E0A90000E2A90000E4A9000097
:10212000E6A90000E8A90000EAA90000EEA9000065
:10213000F0A90000F2A90000F4A90000F01B0020A3
:1021400070200020F8A90000FAA90000FCA90000F6
:10215000FEA9000000AA000002AA000004AA0000D4
:1021600006AA000008AA0000F6A900000AAA0000BA
:102170002DE9F04105460E46144600271148007827
:1021800018B112202070BDE8F0812878012808D00D
:10219000022807D0032802D0042804D100E000BFA1
:1021A00000BF00BF02E001202070ECE700BFFEF797
:1021B00079F807466E613846FEF778F800202070FF
:1021C00000BFE0E72100002010B500F019F801F091
:1021D00081FA01F0ADFA01F0CDFA01F04BFA01F00D
:1021E0000BFA01F061FB01F08BFB01F003FB01F046
:1021F00029FB00F0D1FF00F01FF8FFF70BFF10BD27
:102200000948802102E0491E002204C00029FAD1B9
:10221000064A074B1A601A46126822F007021A6033
:102220000022044B1A807047B0200020B02200200A
:102230006C000020700000207047000010B50024E2
:10224000FEF730F8044608480078012808D107480E
:102250000078FF2804D205480078401C0349087024
:102260002046FEF723F810BD2E000020210000209C
:1022700010B500241A480078012830D1FEF712F872
:1022800004461848007820B116480078401E1549C9
:10229000087014480078F8B913480078E0B901F0E4
:1022A00091FB12481249097850F821001149086041
:1022B0000F4800781049097888420DD00D48006811
:1022C000C06B401C0B490968C8630C480068401C7F
:1022D0000A490860FEF706F82046FDF7E7FF10BD43
:1022E0002E00002021000020220000208812002063
:1022F000240000203C0000202300002008000020D3
:102300002DE9FC5F05460F4691469A460020009055
:10231000FDF7C8FF009018480468006820B116480F
:1023200000684068144908600098FDF7BFFF2CB9A9
:102330005A208AF800000020BDE8FC9FA8462E46DF
:10234000781E01904FF0000B05E04E44C8F8006085
:10235000B0460BF1010B01988345F6D30020C8F875
:102360000000256065602761E760C4F808908AF87E
:1023700000002046E0E70000480000202DE9F04181
:1023800004460D460027FDF78DFF0746206968B11A
:102390006668306860602069401E20613846FDF73D
:1023A00085FF002028703046BDE8F0813846FDF7F3
:1023B0007DFF5D2028700020F6E770B504460D46CD
:1023C0000026FDF76FFF0646D4E90310884204D3C8
:1023D0003046FDF76BFF5E2070BD60682860656069
:1023E0002069401C20613046FDF760FF0020F3E7C4
:1023F0002DE9F04106460F464FF0000820480078CE
:1024000010B10020BDE8F081FDF74CFF80461D486B
:102410000468006820B11B480068406819490860DA
:102420004046FDF743FFFCB1FDF73CFF80461648F0
:102430000568D5B100680068134908604046FDF79B
:1024400035FF6E6006EB8700A860EE602E61AF82FC
:102450000020E882022020700020208165600BA00F
:102460006061204601F0BAF808E006480068606044
:10247000044804604046FDF719FF00242046C1E7E8
:10248000210000200C0000204C0000203F00000034
:102490002DE9F0470746884615464FF00009387881
:1024A000022804D0012028700020BDE8F0873E48B3
:1024B000007818B1022028700020F6E73B48007829
:1024C00018B10D2028700020EFE7FDF7EBFE8146E4
:1024D0007C68E08A98B12169081D20610E68E08A55
:1024E000401EE082A1682069884201D160682061B5
:1024F0004846FDF7DBFE002028703046D5E72C4823
:10250000006890F8340040F004002949096881F817
:10251000340000202649096881F835002448006805
:10252000C0F83080384601F01BF84846FDF7BEFE83
:1025300001F00EFAFDF7B6FE81461D48006890F8DE
:10254000350020B101280DD002280AD105E0184835
:102550000068466A002028700DE000260E202870D2
:1025600009E000BF39461248006800F0C5FF0026A8
:102570000A20287000BF00BF00200D49096881F8BB
:1025800034000B49096881F8350009490968C861B8
:102590000749096808620649096848624846FDF724
:1025A00085FE304681E70000210000202200002047
:1025B000340000202DE9F04105460E46002728781A
:1025C000022802D00120BDE8F081FDF76BFE07462E
:1025D000A87A60B1002304223146284600F044FF67
:1025E0003846FDF763FE01F0B3F90020EBE76C68B5
:1025F000E08AA18A884204DB3846FDF757FE1E2098
:10260000E1E7E168081DE0600E60E08A401CE082BE
:10261000D4E90210884201D16068E0603846FDF7D5
:1026200045FE0020CFE72DE9F04705460C464FF068
:10263000000A2878022802D00120BDE8F087FDF7C3
:1026400031FE8246A87A207405F10B0804F10809CE
:10265000002705E018F8010B09F8010B781CC7B238
:10266000082FF7D36E68F08A18B1306900682060CF
:1026700001E000202060F08AA080B08AE08050460F
:10268000FDF714FE0020D8E710B500240B480078B1
:10269000012811D1FDF706FE04460948007840B92B
:1026A00008480078FF2804D206480078401C0549F5
:1026B00008702046FDF7FAFD10BD00002E00002036
:1026C000210000202200002010B5002413480078CB
:1026D000012821D1FDF7E6FD044611480078C0B974
:1026E0001048007888B10F480078401E0D490870E6
:1026F0000846007828B92046FDF7D8FD01F028F9F2
:102700000AE02046FDF7D2FD06E02046FDF7CEFDAB
:1027100002E02046FDF7CAFD10BD00002E0000209B
:10272000210000202200002070B505460026104838
:10273000007808B1002070BDFDF7B4FD06460D48D5
:102740000468006820B10B480068406809490860C7
:102750003046FDF7ABFD4CB10320207025810020F1
:10276000606005A06061204600F038FF2046E2E787
:10277000210000200C0000203F0000002DE9F04166
:1027800005460E46144600272878032803D001206A
:102790002070BDE8F0813248007810B1022020702E
:1027A000F7E73048007810B10D202070F1E7FDF711
:1027B00079FD0746288940B12889401E288138467E
:1027C000FDF774FD00202070E3E72748006890F8CB
:1027D000340040F001002449096881F834000020E9
:1027E0002149096881F835001F48006806632846BA
:1027F00000F0B6FE3846FDF759FD01F0A9F8FDF7E7
:1028000051FD07461848006890F8350020B10128AE
:1028100009D0022806D102E0002020700BE00E2033
:10282000207008E000BF29460F48006800F064FEF1
:102830000A20207000BF00BF00200B49096881F802
:1028400034000949096881F8350007490968C861F9
:102850000549096808623846FDF728FD00BF98E77A
:1028600021000020220000203400002070B5044622
:1028700000252078032801D0012070BDFDF712FD4E
:102880000546A07A60B1002301221946204600F0D7
:10289000EBFD2846FDF70AFD01F05AF80020ECE7B1
:1028A00020894FF6FF71884207D22089401C208181
:1028B0002846FDF7FBFC0020DFE72846FDF7F6FC85
:1028C0003320DAE710B50B48007890B901F07AF8B8
:1028D000094800780949087009480749097850F8FB
:1028E0002100084908600846006807490860FDF7AC
:1028F000E0FC10BD2E00002024000020230000205A
:10290000881200203C0000203400002010B5002474
:10291000022000F035FBFDF7C5FC044600200B4902
:1029200008602046FDF7C2FC642000F029FBFDF79B
:10293000B9FC0446054800680549086001200549BE
:1029400008702046FDF7B2FC10BD000030000020EA
:10295000180000202000002010B504462046FDF796
:1029600025FE10BD2DE9F04F85B081468A4693467D
:102970001C46DDE90F78129D00200390FDF792FCC4
:1029800003902348007830B10398FDF78FFC3C207A
:1029900005B0BDE8F08F1F4850F8240088BB012027
:1029A0001C4941F824000398FDF780FC2A46414663
:1029B000384601F04BF92B465A465146484600F03E
:1029C00073F904901198CDE9008002953A462046AB
:1029D0000E9B049901F00CF8064636B90E480078B3
:1029E00001280CD100F0B4FF09E0FDF75BFC039077
:1029F0000020084941F824000398FDF757FC3046B1
:102A0000C6E7FFE70398FDF751FC2820C0E7000068
:102A100021000020881200202E00002010B504465E
:102A20002046FDF7C4FD10BD2DE9F0410546002705
:102A30004A48007810B14020BDE8F0813F2D01D117
:102A40003E20F9E7FDF72EFC0746FF2D03D1444851
:102A5000006890F83650434850F8254024B938466D
:102A6000FDF724FC4320E7E7012C04D13846FDF7AD
:102A70001DFC3D20E0E714F8380F3B49085C617805
:102A800088432178384A505414F838091146085CB4
:102A900030B994F83A1035480078884333490870C3
:102AA000E06918B12046E16900F026FD206A18B1FE
:102AB0002046216A00F037FDA66A16B1304600F0C4
:102AC000C7FD0020206384F8340084F835002848CE
:102AD0000078FF2804D226480078401C244908705A
:102AE0003846FDF7E3FB00F0BDFCFDF7DBFB0746D6
:102AF0001F48007820B11E480078401E1C4908700D
:102B0000204600F041F81B480078401E1949087023
:102B10000020144941F82500A06930B900206169FE
:102B2000886115496069086005E0D4E905014861DC
:102B3000D4E9051088611148006860610F4804609D
:102B40000FA020653846FDF7B1FB0E48007801283C
:102B500001D100F0FDFE00206EE700002100002002
:102B600034000020881200202600002025000020CC
:102B7000220000202F00002040000020380000200C
:102B80003F0000002E00002010B504462046FDF74F
:102B90000FFD10BD10B5FDF70CFD10BD2DE9F04186
:102BA00006460F4614464FF000081548007818B145
:102BB00012202070BDE8F081FDF774FB8046FF2EE7
:102BC00003D11048006890F836600F4850F826503E
:102BD0002DB94046FDF76AFB43202070EAE7012D3E
:102BE00005D14046FDF762FB43202070E2E72F65E8
:102BF0004046FDF75BFB0020207000BFDAE70000D5
:102C000021000020340000208812002010B5044666
:102C10002046FDF7CFFC10BD10B5FDF7CCFC10BD74
:102C20002DE9F04707460D464FF0000A00202860C6
:102C30006860FDF737FB8246FF2F03D11848006814
:102C400090F83670174850F827402CB95046FDF7D9
:102C50002DFB4320BDE8F087012C04D15046FDF741
:102C600025FB4320F6E7207C00F0010020B9504608
:102C7000FDF71CFB4520EDE70026D4F80C90D4F8B6
:102C800008805046FDF712FB00E0761C58F8041B44
:102C90000029FAD02E60A9EB060068600020D9E771
:102CA000340000208812002070B50446101D20F06A
:102CB00007004FF08076051F28462E60051F284626
:102CC0002C60684E051F28462E604FF01236051FF7
:102CD00028462E604FF00336051F28462E604FF021
:102CE0000236051F28462E607610051F28462E60E6
:102CF000051F284629604FF01136051F28462E6013
:102D00004FF01036051F28462E604FF00936051F7C
:102D100028462E604FF00836051F28462E604FF0DB
:102D20000736051F28462E604FF00636051F284639
:102D30002E604FF00536051F28462E604FF00436F2
:102D4000051F28462E6003F00405002D7ED0F605F1
:102D5000051F28462E60444E051F28462E60434E10
:102D6000051F28462E60424E051F28462E60414E04
:102D7000051F28462E60404E051F28462E603F4EF8
:102D8000051F28462E603E4E051F28462E603D4EEC
:102D9000051F28462E603C4E051F28462E603B4EE0
:102DA000051F28462E603A4E051F28462E60394ED4
:102DB000051F28462E60384E051F28462E60374EC8
:102DC000051F28462E60364E051F28462E604FF000
:102DD0008346051F28462E60324E051F28462E606A
:102DE000314E051F28462E60304E051F28462E60A6
:102DF0002F4E051F28462E602E4E051F28462E609A
:102E00002D4E051F28462E602C4E051F28462E608D
:102E10004FF08246051F28462E60294E051F284682
:102E20002E60284E051F28462E60274E051F284677
:102E30002E604FF08146051F28462E60234E051F49
:102E400028462E603602051F284600E009E02E6065
:102E50004FF07E56051F28462E600026051F284687
:102E60002E6070BD593B00000000F8410000F041A9
:102E70000000E8410000E0410000D8410000D041DE
:102E80000000C8410000C0410000B8410000B0414E
:102E90000000A8410000A0410000984100009041BE
:102EA0000000884100007041000060410000504176
:102EB000000040410000304100002041000010416E
:102EC0000000E0400000C0400000A0400000404082
:102ED0002DE9F04105464FF00008FDF7E3F9804683
:102EE000FF2D05D12048006890F83650012608E0F3
:102EF0001D48006890F83600A84201D1012600E084
:102F000000261A4850F825402CB94046FDF7CEF966
:102F10004820BDE8F081012C04D14046FDF7C6F9F8
:102F20004320F6E794F838701148C05D94F83910E2
:102F300088430F49C8550846C05D30B994F83A1027
:102F40000C48007888430B49087094F8340040F02E
:102F5000080084F834004046FDF7A8F9012E01D19D
:102F600000F0F6FC0020D4E7340000208812002096
:102F7000260000202500002010B5FDF71DFB10BD28
:102F800070B5054600261748007800B170BD164898
:102F9000007800B1FAE71DB3FDF784F9064613483F
:102FA000006890F838401248005D1049096891F8AF
:102FB000391088430E4908550846005D40B90B4852
:102FC000006890F83A100B48007888430949087067
:102FD0000648006805633046FDF768F900F0B8FC64
:102FE00000BFD3E721000020220000203400002091
:102FF00026000020250000202DE9F04105460E4660
:1030000017461C461248007810B15520BDE8F081E3
:103010001048007808B13220F8E74FF47A70604326
:103020004FF47A71B0FBF1F14FF461606843C6EB85
:10303000061200EB8200384400EB4002C2EBC010E5
:1030400001EBC0084046FFF79BFF0020DEE70000D1
:10305000210000202200002070B50025FDF722F994
:103060000546034804682846FDF720F9204670BD50
:103070005400002070B5002600F072F8FDF712F938
:10308000064631480068401C2F4908603046FDF76D
:103090000DF92E480078012853D12D48007820B131
:1030A000012804D0022809D103E001250BE0002506
:1030B00009E0012501202649087004E001250020CF
:1030C0002349087000BF00BF05B970BD21480468DE
:1030D00033E0FDF7E7F80646206B50B3206B401E47
:1030E0002063206B28BB94F8340000F0370040B117
:1030F00014F8340F00F0C800207001206070343CD8
:1031000002E0002084F8350094F8340000F0080054
:1031100078B93834A0781049097808430E49087006
:1031200020780E49085C6178084314F838190B4A76
:10313000505464693046FDF7B9F894F836003F28DA
:10314000C7D100BFC1E70000540000202E000020BE
:103150004400002040000020250000202600002020
:1031600010B5FDF72AFA06480088401C044908807B
:103170000846008818B10020088000F003F810BD50
:103180007000002010B503480068FFF76FFB04468D
:10319000204610BD64000020F8B54FF42071284887
:1031A00000F078FB4021274800F074FB002514E074
:1031B000681C86B205EB8500214901EBC00406EBD3
:1031C000860001EBC00764202070002084F82500F1
:1031D000E7601DA02062681C85B20F2DE8D305EBC7
:1031E0008500174901EBC00464202070002084F89A
:1031F0002500E06014A020620020144908601449F2
:1032000008801020134908800D48134908600120E8
:10321000FFF78AFA114908600020FFF785FA104984
:1032200008606A460FA10D480068FEF7A1FF6A46D4
:1032300011A10B480068FEF79BFF00F027F8F8BDCE
:10324000F01B0020702000203F0000005C000020E8
:103250005A00002058000020680000206000002074
:103260006400002075432F4F532D494920546D723F
:103270004C6F636B0000000075432F4F532D49497D
:1032800020546D725369676E616C000000B587B0A1
:103290000320002180220A4BCDE90132CDE9031041
:1032A0004FF6FD703D23074A00900748FFF75AFB91
:1032B00006AA06A13D20FFF771FC07B000BD000083
:1032C000701E00206C2000204933000075432F4FF2
:1032D000532D494920546D720000000070B50B4613
:1032E000032580F82550012B05D1154EC569366898
:1032F000354445610CE085692DB9114EC5693668C4
:103300003544456104E00E4E8569366835444561B3
:10331000057D05F007040B4D05EBC4010D682DB9C3
:1033200008600025C56001258D8006E00A680860F8
:10333000C26010618D886D1C8D800025056170BD97
:103340005C0000207020002008B500BF00BF6A4666
:1033500000211A480068FFF711FAFFF795F918489D
:103360000068401C164908600846007800F007080D
:10337000144800EBC8073C681AE0E6681049606929
:103380000968884213D1204600F01EF894F8240002
:10339000022804D101212046FFF7A0FF02E002200D
:1033A00084F82500656815B12046A168A847344611
:1033B000002CE2D1FFF788F9C9E700006400002083
:1033C0005C0000207020002030B5057D05F007046A
:1033D0000D4D05EBC4031D68854205D1C168196018
:1033E00039B100250D6104E00169C268CA6002B10B
:1033F0001161012580F825500025C56005619D8873
:103400006D1E9D8030BD00007020002010B5FCF7BF
:1034100049FF044606480078401C054908702046CC
:10342000FCF744FFFFF726FEFEF722FF10BD000069
:103430002100002001464A1E4FF0E0235A61084A4D
:10344000106820F07F4000BF10601A46126942F0F9
:1034500005021A611A46126942F002021A617047A7
:1034600020ED00E0704700002DE9F04F05460F46C3
:1034700090469946A87A1C490E5C05F10B00805DC8
:1034800011F800B00BEBC60000F0FF0A174850F827
:103490002A4000202434E0602760207C20EA0800D5
:1034A000207484F81190207C243C00F0080068B956
:1034B00094F83A000E49097808430D4908700D4800
:1034C000805D94F8391008430A49885529462046FA
:1034D00000F012F8206A20B12046216A00F023F89B
:1034E000E5615046BDE8F08F98A8000088120020E2
:1034F000250000202600002010B590F8382001F1AA
:103500000B039B5C90F83940A34301F10B04A354D7
:1035100023469B5C23B98B7A90F83A40A3438B7285
:103520000023C36110BDF0B5024612F8384F9578FC
:103530005678383A0B4618680FE000F10B073F5DEC
:10354000B74300F10B0C0CF8047067463F5D17B9E8
:10355000877AAF4387721B1D18680028EDD1F0BD34
:1035600010B51B4A1268D061194A126892F83830B7
:1035700000F10B02D25C164B1B6893F839301A43EA
:10358000134B1B6893F8384000F10B031A55827AED
:103590000F4B1B6893F83A301A4382720C4A126838
:1035A00092F838100B4A525C094B1B6893F839307B
:1035B0009A43084B5A541A46525C42B9044A12685C
:1035C00092F83A30044A12789A43034B1A7010BDAD
:1035D00034000020260000202500002001460022A3
:1035E0008A72002005E0002301F10B021354421CF3
:1035F000D0B20828F7D370472DE9F041A021114837
:1036000000F048F900250DE0681C86B20D4800EB7B
:10361000051400EB06170020207067600AA0E06028
:10362000681C85B2092DEFD3064800EB0514002075
:103630002070606004A0E060024804490860BDE8B2
:10364000F0810000E80D00203F0000001000002085
:1036500030B501464A6808682AB9CC68606028B16C
:103660000025456002E0106000B142608B680025D3
:103670009D6230BD70B54FF4C061134800F00AF987
:10368000002411E0601C85B204EB44000E4901EBFC
:10369000C00305EB450001EBC006002018705E601A
:1036A0000AA05861601C84B23F2CEBD304EB4400A9
:1036B000054901EBC00300201870586003A0586151
:1036C00008460349086070BDE80700203F0000007D
:1036D0000C00002000200B4908600B4908700B49C2
:1036E00008700B4908700B4908700B4908600B49BA
:1036F00008600B4908600B4908600B4908700B49CA
:103700000870704754000020210000202200002093
:103710002F0000202E000020080000203000002094
:103720001C00002018000020200000205000002075
:1037300000210A4A1170002004E00021084A1154B7
:10374000411CC8B20828F8D30021064A1170064A65
:103750001170064A1160064A11607047250000206A
:103760002600002023000020240000203C00002030
:103770003400002070B54FF4F261194800F08AF867
:103780004FF48071174800F085F8002413E0601CA6
:10379000C5B204EB440000EBC400114901EBC003C7
:1037A00005EB450000EBC50001EBC0065E610EA015
:1037B0001865601CC4B2152CE9D304EB440000EB7F
:1037C000C400074901EBC0030020586106A018653A
:1037D00000200649086002480549086070BD0000E5
:1037E00088130020881200203F00000040000020C5
:1037F0003800002000B587B00320002180220A4B4A
:10380000CDE90132CDE903104FF6FF703F23074A9F
:1038100000900748FFF7A6F806AA06A13F20FFF789
:10382000BDF907B000BD0000881000208412002000
:10383000313B000075432F4F532D49492049646C9B
:103840006500000000B587B00320002180220A4BEC
:10385000CDE90132CDE903104FF6FE703E23074A51
:1038600000900748FFF77EF806AA06A13E20FFF762
:1038700095F907B000BD0000880E002084100020DC
:10388000713B000075432F4F532D494920537461FC
:103890007400000004E0002200F8012B4A1E91B2DF
:1038A0000029F8D17047000070B578211148FFF762
:1038B000F1FF00240EE004EB44000E4901EBC005CB
:1038C000601C00EB400001EBC00068600AA068616A
:1038D000601C84B2042CEED304EB4400054901EBD8
:1038E000C0050020686004A06861084603490860BC
:1038F00070BD0000181B00203F00000048000020A1
:103900002DE9F04160211048FFF7C4FF00240DE0CD
:10391000601C86B204EB44000B4901EBC00506EBCA
:10392000460001EBC0072F60601C84B2032CEFD36C
:1039300004EB4400044901EBC00500202860084660
:1039400002490860BDE8F081901B00204C00002077
:1039500010B50024FCF7A6FC044613480078F8B91B
:1039600012480078E0B900F02DF8114811490978A3
:1039700050F82100104908600E4800780F49097876
:1039800088420DD00C480068C06B401C0A49096889
:10399000C8630B480068401C09490860FCF79DFC9F
:1039A0002046FCF783FC10BD2100002022000020EF
:1039B00088120020240000203C000020230000206A
:1039C000080000200649074A1278885C0649095C0D
:1039D000034A515C01EBC001044A117070470000BA
:1039E00098A80000250000202600002024000020C8
:1039F0002DE9F84F05460F4690469946DDE90AAB9A
:103A000000200090FCF74EFC009042480468002C17
:103A10007BD01C3454F8080C3E4908600098FCF731
:103A200045FC44F81C7CA576002020766076606119
:103A300044F818BC44F810AC44F8148C0C9824F8E2
:103A40000C0C24F80A9C0020E077E810207705F0A1
:103A50000700E076217F01208840A077E17E0120E9
:103A600088406077002020606060E060A060206295
:103A7000A0626062E062206327A060631C3C0026B5
:103A800006E0002104F1540040F82610701CC6B274
:103A9000002EF6D02046FEF75FFFFCF703FC0090F7
:103AA0001E4840F825400098FCF700FC2046FEF731
:103AB000B5FFFCF7F7FB0090194800686061002033
:103AC000A0611748006810B1154800688461144867
:103AD00004603834A0781349097808431149087004
:103AE00020781149085C6178084314F838190E4AA7
:103AF00050540E480078401C0C4908700098FCF7A0
:103B0000D5FB0020BDE8F88FFFE70098FCF7CEFB5F
:103B10004220F7E7380000203F0000008812002014
:103B20004000002025000020260000202F0000205B
:103B3000002400BF00BFFCF7B5FB04460548006841
:103B4000401C044908602046FCF7B0FBFFF722F850
:103B5000F1E700003000002010B504480068FFF7CE
:103B600055F8FF20FEF760FF10BD00003400002074
:103B700000BF00BF02E0C820FFF702FA1F4800782C
:103B80000028F8D01E4800686421B0FBF1F01C4901
:103B900008600846006828B900201A490870FF200C
:103BA000FFF796F9FCF77EFB044615480068642190
:103BB0004843154908602046FCF778FB00BFFCF736
:103BC00071FB0446104800681049086000200E4947
:103BD00008602046FCF76AFB0C4800680849096841
:103BE000B0FBF1F0C0F1640006490870FFF714F86B
:103BF00000F00EF86420FFF7C3F9E0E72000002092
:103C00001800002014000020300000201C000020BC
:103C10007CB5002514E069462846FFF701F8064602
:103C200066B9094850F8254044B1012C06D0D4E9C2
:103C3000020100EB8100A0640198E064681CC5B239
:103C40003F2DE8D97CBD00008812002002F001035E
:103C500043B102F002032BB102E0491E002308C069
:103C60000029FAD1704700002DE9FC4104460D46B9
:103C70001646019400200090012301AA68211548EE
:103C80000078FDF7A1F807463846FDF705FC002847
:103C900003DA4FF0FF30BDE8FC8101236A4668215A
:103CA0000C480078FDF702F807463846FDF7F4FBAC
:103CB000002802DA4FF0FF30EDE79DF8000000F039
:103CC0000F013040001100EB800001EB4000287034
:103CD0000020E0E7AC01002008E00548FDF7E4FB28
:103CE0000023012219461846FFF786F9F5E7000080
:103CF000C8010020F8B504460D468DF800408DF847
:103D0000015002236A46682103480078FDF75CF8F9
:103D10000646FDF7C1FBF8BDAC01002070B50446B6
:103D20000D4616460CB9002070BD0DB90020FBE70A
:103D300021462A46002304E010780870491C521CD2
:103D40005B1C21B11AB1107808B1B342F4D301B1B0
:103D50000AB90020E8E7B34201D2002008702046EB
:103D6000E2E710B502460B461146002001E0491C6F
:103D7000401C19B10C780CB19842F8D310BD00006A
:103D800010B50121C0F30722094B1A4402F070421A
:103D900042F00072C0F30723054C2344C3F313031E
:103DA00042EA4312C3B242EA8302116010BD00002E
:103DB00000E60F400146C1F307200B4A104400F013
:103DC000704040F00070C1F30722074B1A44C2F361
:103DD000130240EA4210CAB240EA8200006808B109
:103DE000012070470020FCE700E30F400146C1F3CB
:103DF00007200B4A104400F0704040F00070C1F3FF
:103E00000722074B1A44C2F3130240EA4210CAB217
:103E100040EA8200006808B1012070470020FCE7FA
:103E200000EA0F4018B50121C0F30722184B1A44CD
:103E300002F0704242F00072C0F30723144C234496
:103E4000C3F3130342EA4312C3B242EA830211608E
:103E50000021009102E00099491C0091009910296D
:103E6000F9D30021C0F30722094B1A4402F0704233
:103E700042F00072C0F30723054C2344C3F313033D
:103E800042EA4312C3B242EA8302116018BD000045
:103E900000E50F400146886900F0100008B9086885
:103EA00070474FF0FF30FBE700BF826902F020024D
:103EB000002AFAD10160704701468869012222EA8E
:103EC00010107047F0B504460E4615461F462046B2
:103ED00000F01EF8B6EB051F05D2206B40F0200065
:103EE00020636D0803E0206B20F020002063F000C9
:103EF000B0FBF5F0401C43089809606203F03F00F6
:103F0000A062E7620020A061204600F011F8F0BD39
:103F100000BF816901F008010029FAD1C16A21F0CE
:103F20001001C162016B40F201329143016370479D
:103F3000C16A41F01001C162016B40F201321143CC
:103F40000163704741647047826B0A438263704724
:103F5000024609B1106C7047D06BFCE72DE9F84FB1
:103F600080460C4615461E46DDF84CB0DDE90C9A3D
:103F70000E9F4046FFF704FF2046FFF701FF0A9817
:103F8000FDF71AFE0B98FDF717FE49EA0A00C1B2C9
:103F90003046FDF766FEFCF74FFE0090129840EAAF
:103FA0000B00149940EA01032846119A0099FFF783
:103FB00089FFF8B20F99FCF771FDF8B2FCF704FB2A
:103FC0001098FDF76BFF60211098FDF7A9FF5021B5
:103FD0002846FFF7B9FF0020BDE8F88F1FB51BE0AA
:103FE0000E48407800900D488378C2780CA101A853
:103FF00000F08EF8002405E001A8015D0C48FFF7F1
:1040000053FF641C01A8005D0028F5D100230122A4
:1040100019461846FEF7F0FFE2E70000C80100204D
:10402000253032753A253032753A25303275000028
:1040300000D000407FB588B0DDE91045E0B28DF8D2
:1040400018004FF47F4104EA01000021000A40EA11
:104050000160C0B28DF819004FF47F0104EA01003D
:104060000021000C40EA0140C0B28DF81A004FF068
:104070007F4104EA01000021000E40EA0120C0B2A5
:104080008DF81B00E8B28DF81C004FF47F402840EB
:10409000000A8DF81D009DF8200000069DF82110F3
:1040A00040EA01409DF8221040EA01209DF82310CB
:1040B000084305909DF8240000069DF8251040EA6D
:1040C00001409DF8261040EA01209DF82710084382
:1040D00004909DF8280000069DF8291040EA014050
:1040E0009DF82A1040EA01209DF82B100843039008
:1040F000FCF7A2FD064600210398CDE9000106A9C0
:104100003046DDE9043201F07DFA0CB070BD0000EC
:104110000FB4084B10B504A902AA039800F01CF8CC
:10412000044602A9002000F0B8F9204610BC5DF852
:1041300014FB00009B44000002E008C8121F08C1E5
:10414000002AFAD170477047002001E001C1121F18
:10415000002AFBD1704700002DE9FF4F8BB0884645
:104160000546002606E025280BD0DDE90D12904714
:104170006D1C761C28780028F5D10FB03046BDE8BC
:10418000F08F0024A146A2460122AE4900E004437C
:1041900015F8013F203B02FA03F00842F7D12878D6
:1041A0002A2810D06FF02F022878A0F130010929B9
:1041B00015D809EB890102EB410144F0020400EB40
:1041C00001096D1CF0E758F8041B5FEA010903D5EB
:1041D00044F40054C9F1000944F002046D1C28782D
:1041E0002E2817D115F8010F44F004042A280ED008
:1041F0006FF02F022878A0F1300109290AD80AEBC4
:104200008A0102EB410100EB010A6D1CF2E758F84C
:1042100004AB6D1C28786C280FD006DC4C2817D016
:1042200068280DD06A2814D104E0742810D07A28A8
:104230000FD10DE044F400140AE044F4801401E0CE
:1042400044F440146978814202D104F580146D1C55
:104250006D1C2878692865D006DC00288DD063287D
:1042600027D0642806D15DE06E2808D073282AD0B4
:10427000752877D0DDE90D129047761CE0E0C4F395
:104280000250022809D003280DD0D8F800100428C5
:104290000DD00E6008F10408D2E0D8F80010F21733
:1042A000C1E90062F6E7D8F800100E80F2E70E7060
:1042B000F0E718F8041B8DF8001000208DF80100BD
:1042C000EB46012003E058F804BB4FF0FF306107D4
:1042D0004FF0000701D40AE07F1C57450DDA8742F2
:1042E000FADB1BF807100029F6D106E07F1C874295
:1042F000FCDB1BF807100029F8D1DDE90D23A9EB41
:1043000007008146214600F0B1F83044C61904E0A8
:10431000DDE90D121BF8010B90477F1EF8D22146F4
:10432000484688E058F8040BC4F302514FF00A0BDA
:10433000032900D100B2042900D140B2002802DADA
:1043400040422D2102E0210505D52B218DF82410B6
:10435000012104E006E0E10710D02021F6E708AFD4
:10436000089113E058F8040BC4F302514FF00A0B04
:10437000032900D180B2042900D1C0B20021EEE7A8
:104380005946FCF752F8303107F8011D0028F7D1E3
:10439000ADEB070000F1200B600702D524F4803458
:1043A00001E04FF0010ADA4502DDAAEB0B0000E064
:1043B0000020824600EB0B0108980144A9EB0100A4
:1043C0000A90E00306D4DDE90D2321460A9800F0A7
:1043D0004DF806444FF0000908E009A911F809005A
:1043E000DDE90D12904709F10109761C089989450C
:1043F000F3DBE0030CD5DDE90D2321460A9800F03C
:1044000035F8064404E0DDE90D1230209047761CB3
:10441000BAF10001AAF1010AF5DC05E0DDE90D12AF
:1044200017F8010B9047761CBBF10001ABF1010BB3
:10443000F4DC0A982146DDE90D2300F005F8064476
:104440006D1C97E6092801002DE9F041044600257E
:104450001E461746880404D405E039462020B0479C
:104460006D1C641EF9D52846BDE8F0812DE9F041A8
:10447000044600251E469046C80301D5302700E0BB
:104480002027880404D505E041463846B0476D1C16
:10449000641EF9D52846BDE8F0810A68531C0B60FC
:1044A0001070704710B5044600F0FCFB0022034971
:1044B00041F2883002F098FB10BD0000A5440000D6
:1044C00010B50446A4B91748FFF75AFC1648FFF781
:1044D00057FC1648FDF770FB1548FDF76DFB0421EE
:1044E0001448FDF7AFFB08211248FDF79CFB17E0CD
:1044F000012C15D10B48401CFFF742FC0A48401D17
:10450000FFF73EFC0C48FDF757FB0C48FDF754FB4A
:1045100001210B48FDF796FB02210948FDF783FBBB
:1045200010BD0000002000F0010800F002080100AA
:10453000020C0100005000400200060002040600C8
:10454000006002402DE9FC4705468846164600BF3C
:104550000DB9BDE8FC8700BF70892A280EDA4B48E8
:10456000408C401C81B249484184C08B401C81B2C0
:104570004648C183304602F04DF8EAE7776807F114
:104580000E042088B0F5807F08D12079062805D157
:104590006079042802D1608808280ED03B48008D3D
:1045A000401C81B239480185C08B401C81B237481C
:1045B000C183304602F02EF8CBE73448408B401CD4
:1045C00081B232484183D4F80E000190A069009076
:1045D000281D08B1686810B94FF0000907E000987D
:1045E0006968884201D1012000E000208146B9F1CC
:1045F000000F01D0012000E00220034604F1080270
:1046000001A9284600F094FBE088B0F5807F03D034
:10461000B0F5007F2DD12BE0B9F1000F26D002209C
:1046200001F0ADF8E080D4F80E00A0616868C4F82D
:104630000E0000BF00BFA068C4F81200A089E0828D
:10464000A0683860A089B880D8F80000A060B8F8E9
:104650000400A081D8F80000C7F80600B8F80400EC
:10466000788131462846AA69904700E000BF07E0FC
:1046700006E00648808D401C81B20448818500BF59
:1046800000BF304601F0C6FF00BF62E7B8F500206A
:104690002DE9FC5F05460F464FF00A08C1460A2681
:1046A0000024A34600200190B246009000BF5CE0C9
:1046B00004EB84004D4A02EB8000817C0A2E02D17B
:1046C00009B966B24FE000294DD000BF00BF5DB10F
:1046D00004EB8402454B03EB820228685268904247
:1046E00002D160B2BDE8FC9F012928D104EB84000F
:1046F0003E4A52F8200088B104EB840002EB8000AF
:10470000C27C009882422EDB4FFA84FA04EB8400CC
:10471000364A02EB8000C07C009024E004EB840069
:10472000324A02EB8000C07C58451CDB4FFA84F80B
:1047300004EB840002EB800090F813B013E0022930
:1047400011DB04EB8400294A02EB8000C27C019853
:10475000824208DB4FFA84F904EB8400234A02EB1F
:104760008000C07C0190601CC4B20A2CA0DB07F062
:10477000020020B90A2E05D107F0010010B94FF050
:10478000FF30AFE70A2E01DAF4B21AE0B9F10A0FEE
:1047900003DA09F0FF0400BF0EE0B8F10A0F02DAF5
:1047A00008F0FF0408E0BAF10A0F02DA0AF0FF0489
:1047B00002E04FF0FF3095E700BF00BF204600F059
:1047C00017F800BF00BF00BF00BF35B104EB840184
:1047D000064A02EB810128684860002004EB84014E
:1047E000024A02EB8101C87460B27BE7ECF600205C
:1047F00010B5044604EB84000C4951F8200060B168
:1048000004EB8401094A52F8210001F003FF002063
:1048100004EB8401054A42F82100002004EB8401E6
:10482000024A02EB8101887410BD0000ECF6002002
:104830002DE9FC4704460F461546A94600BF00BFB8
:1048400000BF00BF00BF00BF0E21384601F047FF88
:1048500040B14B484089401C494948816FF00100F4
:10486000BDE8FC872146286800F0A3FC10B1DFF802
:1048700014817DE0287800F0F000E02815D10120B7
:104880008DF8000000208DF801005E208DF80200F8
:10489000687800F07F008DF80300A8788DF8040098
:1048A000E8788DF80500E84661E02868A1680840CE
:1048B000D4E901121140884210D0288880B24FF606
:1048C000A96188420AD004F10C0020B1E06810B15F
:1048D00004F10C0902E06FF00300C1E72A480078F8
:1048E00000EB8000294901EB8000807C022818DB66
:1048F0002549097801EB8101244A02EB8101D9F8AD
:104900000000496888420CD11D48C08D401C81B20E
:104910001B48C1851C4802783946204600F038F80B
:104920009EE700261BE006EB8600184901EB80009D
:10493000807C022811DB06EB8601144A02EB810120
:10494000D9F800004968884207D10F490E70F2B2C9
:104950003946204600F01CF882E7701C46B20A2E49
:10496000E1DB3A464946204600F048F878E700BFC8
:10497000434604F12F023946204600F077F96FE7ED
:10498000B8F500208CAB00000A010020ECF60020F6
:1049900070B505460E46144600BF00BF04EB840008
:1049A000154901EB8000807C022817D104EB8400BC
:1049B00001EB8000C07CE42810DB04EB84000A4695
:1049C00002EB8000011D284600F03AF930B90320BF
:1049D00004EB8401084A02EB8101887404EB840033
:1049E000054901EB800000F10C0305F12F0231466F
:1049F000284600F03BF970BDECF600202DE9F05F91
:104A000080460F46164608F12F094FF0FF3A4146FF
:104A1000386800F0CEFB38B9387800F0F000E028B4
:104A200002D00FB1386818B96FF00D00BDE8F09FE3
:104A300001213846FFF72CFE0446002C08DA2EB17F
:104A40004948808C401C81B2474881842046EDE76C
:104A500004EB8400454901EB8000807C30B90120E3
:104A600004EB8401414A02EB8101887400BF00BF5E
:104A700004EB84003D4901EB8000807C012800D0DC
:104A80003EB93946404600F0DBF882460EB9504642
:104A9000CCE700BF00BF04EB8400344901EB800089
:104AA000807C02280FDB32490C7004EB84002F4914
:104AB00001EB800000F10C034A463146404600F00D
:104AC000D5F882464EE004EB8400284901EB8000D3
:104AD000807C012846D14FF0000B354608E000BF2E
:104AE00000BF287B012802D04FF0010B02E02D68A7
:104AF000002DF4D100BFBBF1000F10D02989002296
:104B0000032001F0C7FB05466DB13146284601F090
:104B1000D8FC40B1284601F07DFD002503E0354674
:104B2000284601F07BFEA5B104EB84000F4951F843
:104B3000200030B104EB84010C4A52F8210001F04E
:104B400069FD04EB8400094941F820504FF0000A48
:104B500007E00548808C401C81B2034881844FF0F7
:104B6000FF3A00BF504661E7B8F50020ECF60020A0
:104B70000A0100202DE9F84F0746884691469A46DB
:104B8000DDF828B00020009000BF00BF00222A21DD
:104B9000032001F07FFB05464DB92848808C401C5E
:104BA00081B2264881844FF0FF30BDE8F88F00BF06
:104BB00000BF6E6806F10E040D9800F0E0FDE08085
:104BC00000BF00BFDAF80000A060BAF80400A081BE
:104BD0000B980168C4F812108088E082D9F80000B0
:104BE0003060B9F80400B080D8F80000C6F80600BC
:104BF000B8F804007081DBF80000C4F80E000C98CF
:104C00000068A0614FF4807020800820608006203A
:104C10002071042060714FF4C160B081294638468C
:104C2000BA69904700900548008B401C03490883EF
:104C3000284601F0EFFC00250098B6E7B8F5002003
:104C40007FB504460D460121064A201D04F12F03BD
:104C50008DE825000391044A19462046FFF78AFF94
:104C600004B070BD92AB00008CAB00002DE9F041A8
:104C700005460E4617469846746800BF00BFD8F830
:104C800000002060B8F80400A0803868C4F806006E
:104C9000B88860810820A08131462846AA699047DB
:104CA000BDE8F08170B500243DE004EB84001F49AD
:104CB00001EB8000857C25B304EB840001EB8000D0
:104CC000C07C401C04EB8401184A02EB8101C874CB
:104CD00004EB8400114601EB8000C07CF0280DDA63
:104CE00004EB840001EB8000807C01280AD104EBF6
:104CF000840001EB8000C07C022803DB2046FFF724
:104D000077FD0EE004EB8400084901EB8000807C15
:104D1000032806D1022004EB8401044A02EB81013E
:104D20008874601CC4B20A2CBFDB70BDECF6002096
:104D30002DE9F04706460D461746984600BF00BFCE
:104D40005DB1286848B13146286800F032FA20B9D0
:104D5000287800F0F000E02803D16FF00D00BDE8E6
:104D6000F08741462846FFF793FC0446002C01DA01
:104D70002046F4E7022004EB84011A4A02EB810189
:104D8000887404EB8400114601EB8000866004EB1C
:104D9000840001EB80003968C160B988018200207D
:104DA00004EB840102EB8101C87404EB840011461A
:104DB00051F8200098B104EB840051F820900020B5
:104DC00004EB840142F821003B4606F12F024946DC
:104DD0003046FFF74BFF484601F01CFC00BF0020A7
:104DE000BDE70000ECF600202DE9F04104460E4638
:104DF0004FF00E0860890E280BDC3348008D401CF4
:104E000081B231480185C08B401C81B22E48C183DC
:104E100054E06568AF89287800F00100B0B12878C7
:104E2000012809D1687888B9A8785E280ED1607BFE
:104E300040F01000607309E0062224492846FBF781
:104E4000E7FA18B9607B40F008006073082F03D0C0
:104E5000B7F5C16F22D114E096F8350000F02000BC
:104E600000B92BE0C8F1000001B2204601F037FC88
:104E700010B100BF00BF21E03146204600F0C0F96C
:104E800018E096F8350000F0200000B916E0224640
:104E900006F12F013046FFF755FB0BE00A48008D65
:104EA000401C81B208480185C08B401C81B2064875
:104EB000C18303E000BF0020BDE8F081204601F07F
:104EC000A9FB0020F8E70000B8F500208CAB00003B
:104ED00070B505460C4622460321284600F0F2F83C
:104EE00070BD00002DE9FE4F044689467248B0F8B7
:104EF0004A00401C81B27048A0F84A1065682878C2
:104F000000074FEA9068C8F10001204601F0E7FB76
:104F100010B92089042800D2B4E0606890F800A09D
:104F2000BAF1000F03D0BAF1080F7DD100E0A4E080
:104F300001266248007800F0F000E02800D1002649
:104F40005E490868494600F034F900B1002666B9A8
:104F50005948B0F85C00401C81B25748A0F85C107A
:104F6000204601F057FBBDE8FE8F2089082800D2BB
:104F700088E0204600F0F2F858B1204601F04AFBE4
:104F80004D48B0F85000401C81B24B48A0F850107A
:104F9000E9E72421204601F0A2FB48B34146204620
:104FA00001F09DFB10B100BF00BF77E02189002216
:104FB000022001F06FF9064606B96FE000BF00BF9E
:104FC0002146304601F07DFA10B100BF00BF65E018
:104FD0007568C8F1000001B2304601F080FB10B1E5
:104FE00000BF00BF5AE0204601F014FB344608E041
:104FF0006FF02301204601F072FB10B100BF00BF2B
:105000004CE067682D480068E8602D48006828611A
:10501000002038707880FF202872002068812648A0
:10502000B0F84800401C00E017E02349A1F8480010
:105030004146204601F053FB08B100BF0CE00120BF
:105040000021FF230A46CDE9010900911B492046B2
:1050500000F0FEF9064600BF0FE01748B0F8580010
:10506000401C81B21448A0F85810B0F84E00401C03
:1050700081B21148A0F84E1000BF00BF204601F0D9
:10508000C9FA70E7204601F0C5FA0B48B0F85200A3
:10509000401C81B20848A0F8521064E7204601F095
:1050A000B9FA0548B0F85C00401C81B20248A0F88B
:1050B0005C1000BF57E70000B8F500200401002095
:1050C000000100202DE9FE4306460F4690460022CF
:1050D0002421012001F0DEF805460DB9BDE8FE836C
:1050E00000BF00BFD6F804906C68277084F8018078
:1050F0000020A080E08071686A6802F108001C222C
:10510000FBF748F9002060806989204600F01CF810
:1051100060800C48B0F84800401C0A49A1F84800DB
:10512000D9F80C00029001200021FF2302AACDE94A
:105130000010284600F068F9284601F06BFA00BF1D
:10514000CCE70000B8F5002070B504460D462946AE
:10515000204600F03BFBC04380B270BD2DE9F0411A
:10516000064600240027354617E06989686800F084
:105170002DFB0444A0B200EB1444688900EBD0710D
:105180004910A0EB410139B1C7F10100C7B2E0B24B
:10519000C4F3072141EA00242D68002DE5D127B191
:1051A000E0B2C4F3072141EA0024E04380B2BDE845
:1051B000F08118B502460092D04300B10AB901202F
:1051C00018BD91F8350000F0020008B90020F7E79B
:1051D0004868904201D10020F2E700988B6818409F
:1051E000D1E901342340984208D1886822EA0000BE
:1051F0008C68E343984201D10120E1E70020DFE71A
:105200002DE9F04706460F467948408E401C81B292
:1052100077484186756828780421B1EB201F12D0A9
:10522000304601F0F7F97248B0F84400401C81B2F2
:105230006F48A0F84410C08E401C81B26C48C186F3
:105240000020BDE8F087287800F00F094FF6FF70C6
:1052500000EA8909688800F0B2FA804670894845FA
:1052600002DB308940450FDA304601F0D3F960485F
:10527000408F401C81B25E484187C08E401C81B285
:105280005B48C1860020DCE74146304601F08AFADF
:10529000286958490860E868574908604FF0010AD2
:1052A0003C4600BF94F8350000F0010078B1201DA5
:1052B00068B1606858B14F4800686168884205D09D
:1052C0004C4908682146FFF774FF00B10DE0BAF1C0
:1052D000000F04D04FF0000A4848046800E024683A
:1052E000BC4200D12468002CDCD100BF42490868D0
:1052F0003946FFF75EFF28B93F48007800F0F0001C
:10530000E0280AD1304601F085F93948C08E401CAA
:1053100081B23748C186002093E724B9304601F0B6
:1053200079F900208DE7E8884FF63F71084088B191
:10533000304601F06FF92E48B0F84200401C81B2AF
:105340002B48A0F84210C08E401C81B22848C1866C
:10535000002076E72A4807602A480560394630462B
:1053600001F0AEFAC0BB687A01280DD0062806D03D
:1053700011280ED13946304604F0D6FF2BE03946CD
:10538000304602F085F826E039463046FFF7AAFDA0
:1053900021E0184908683946FFF70BFF50B9154856
:1053A000007800F0F000E02804D07560022130465B
:1053B000FFF78EFD304601F02DF90D48B0F84000A2
:1053C000401C81B20A48A0F84010C08E401C81B237
:1053D0000748C18600BF00BF00200949086009498D
:1053E0000860054908600349086000BF29E700001C
:1053F000B8F50020040100200001002094000020E6
:10540000F8000020FC0000202DE9FE4F06460F4664
:1054100015469846DDE90C9A00BF00BF284600F00B
:105420007DF8041E08D10948C08F401C81B207488E
:10543000C187201FBDE8FE8F43462A4639463046C5
:10544000CDE9009A029400F003F8F3E7B8F50020E4
:105450002DE9F84F05460E4617469A46DDF828B066
:10546000DDF8308000BF00BF002F43D04FF014099B
:105470001421284601F033F958B12648B0F8440009
:10548000401C81B22348A0F844106FF00100BDE831
:10549000F88F6C6800BF00BF84F808A00B9860729A
:1054A0003868206148464FEAE97109EB9171C1F310
:1054B000870141F04001217084F801B0288900F093
:1054C0005EF960800020E0801348008800F057F902
:1054D000A08011480088401C0F4908800EB1306838
:1054E00018B9D8F80400E06001E03068E0600020FE
:1054F000608103E06C68206900906F460548008E6B
:10550000401C044908863A4629464046D8F81430DB
:105510009847BCE7B8F500200801002010B5024606
:10552000144801680FE091F8350000F0010048B11F
:1055300010688B681840D1E901342340984201D1AA
:10554000084610BD09680029EDD10B48006830B14C
:105550000948006890F8350000F0010038B90748A4
:10556000C08F401C83B20548C3870020E9E702488A
:105570000068E6E79400002098000020B8F50020BD
:1055800070B50025FCF75AFEFAF78CFE054601219E
:105590001848FCF779F9044604F0805050B11548DA
:1055A000FCF71FFA1348FCF706FA1248FCF7EDF96E
:1055B00024F080541CB121460E48FCF727F904F072
:1055C000005058B10B48FCF701FA06460A4800683B
:1055D00020B131460748084A126890471CB121465D
:1055E000064804F00DFC2846FAF760FEFCF740FE82
:1055F00070BD000000C00E4098010020F02A01207C
:10560000704700002DE9FC4704460D4616461F462C
:10561000DDE90A892248FEF7B3FB2148FEF702FCC8
:105620002048FEF7C7FB30B11E48FEF7A9FB1D4816
:10563000FEF7F8FB01E000BFFEE700BF1848FEF7E9
:10564000D5FB0028FAD040F20E411748FCF736F996
:10565000002004210B46154ACDE9001021461248CE
:10566000FCF780F800234FF008724FF440610E48B9
:10567000FCF756F82A4600210B48FCF714F80C48B2
:10568000C0F800900B4806600B4807600B48C0F854
:10569000008000210A4804F0DBF9BDE8FC87000027
:1056A000009C00F0003000F000C00E40020000043A
:1056B0009C010020A0010020A4010020A8010020DE
:1056C000DD56000010B50446FFF79AFF002202499C
:1056D000012001F089FA10BDC556000010B586B052
:1056E00004461848006878B91748006800F03AF88E
:1056F00005901648006800F035F8049014480068DA
:1057000000F030F8039003E000200590049003902F
:1057100010481149002203ABCDE90021029004AAF0
:1057200005A90E4800F0C0FC0C4800F00BFD0B482A
:1057300000F08DFD00220A49012001F055FA06B063
:1057400010BD00009C010020A0010020A401002049
:10575000A8010020B99A0000C19D0000F02A012094
:10576000C55600000146080601F47F4240EA0220C7
:1057700001F47F0240EA122040EA116070470146BE
:105780000806000C40EA1120704710B501F0DAF865
:1057900001F05CF900F0EEF800F0D2FA00F0BCFC89
:1057A00000F013F804F0BEFD01F070FE01F088FA7D
:1057B00010BD00B503461846FFF7D4FF00BD00B585
:1057C00002461046FFF7DBFF00BD7047F8B50546FF
:1057D0000A462B4600200090002103F0010636B156
:1057E000002A04DD13F8010B8DF80100521E1C463F
:1057F00003E034F8027B3944921E012AF9DC002AC6
:1058000002DD20788DF80000BDF80000014488B268
:1058100000EB114188B200EB114126B1C8B2C1F3CF
:10582000072747EA002188B2F8BD000088B006A922
:105830000FA0FBF7D3FDFAF705FDFCF7C5FC03202D
:1058400000214FF480720E4BCDE90132CDE90310F7
:10585000042003460B4A00900B48FDF783F807AA83
:105860000AA10420FDF79AF9FDF72CF800BFFEE726
:10587000544D3443313239344E43504454000000C7
:105880002C2B0120282F0120350500005374617254
:105890007400000070B505460C460C48844208D1DF
:1058A000FBF7CAF90646012231462846FCF70CFAF6
:1058B0000AE00748844207D1FBF7BEF906460022FA
:1058C00031462846FCF700FA70BD0000801A060039
:1058D000A086010070B5054605B970BD00BF00BFC8
:1058E00000BF00BF1E480068854203D31D48006802
:1058F00085420FD3002601F06DF806461A48B0F82D
:105900009800401C81B21848A0F89810304601F069
:1059100097F8E2E70021154801F060F8A5F10804C6
:1059200000BF00BF0020207111480068844201D2EE
:105930000F48046020880A490988611A411A0A48F8
:10594000B0F89200401A81B20748A0F892102046A1
:1059500000F072FF054801F007F900BFBDE7000045
:105960008400002088000020B8F50020900000206E
:105970008C00002010B500BF00BF174820F00300C6
:1059800016490860084604684FF420502080002023
:10599000608020710846006800F5205010490860BA
:1059A0000120096808714FF420500D4909680880EA
:1059B0000B4909684880094800680A4908604FF4A3
:1059C00020500949A1F890000121084801F0B2F8DF
:1059D00008B100BF00BF10BDB3220020840000202A
:1059E000880000208C000020B8F5002090000020E6
:1059F0002DE9F041054615B90020BDE8F081E81C0D
:105A000020F0030085B20C2D00DA0C25B5F5205FDF
:105A100001DD0020F1E70021524800F0DFFF52488D
:105A2000008852490988401A86B289E04F480068C8
:105A30008419207900287CD1218806F10800081AF1
:105A4000A8427AD3218806F10800091A05F114004A
:105A5000814232D306F1080028441FFA80F84348F7
:105A6000006800EB080700203871208838807E80AD
:105A7000A4F80080012020713888B0F5205F05D09F
:105A800038883A4909680844A0F8028000BF3848BD
:105A9000B0F8921005F10800084481B23448A0F82B
:105AA0009210B0F89410B0F89200814204DA3048B5
:105AB000B0F89210A0F894101BE00120207100BFF4
:105AC00020882A490988611A411A2948B0F89200A9
:105AD000084481B22648A0F89210B0F89410B0F8AB
:105AE0009200814204DA2248B0F89210A0F8941093
:105AF00000BF1D480068844211D11B49086803E0BB
:105B000001881A4A12688818017919B11949096877
:105B10008842F5D11449086000BF00BF00BF11489A
:105B200001F022F800BF00BF00BF00BF00BF00BFF0
:105B300000E002E004F108005FE70C480068865BC3
:105B4000C5F52050B0423FF771AF0948B0F8960054
:105B5000401C81B20648A0F89610024801F004F8F3
:105B600000204AE7900000208C00002084000020E4
:105B7000B8F50020880000202DE9F05F82460D4630
:105B8000E81C20F0030085B20C2D00DA0C25B5F5D9
:105B9000205F02DD0020BDE8F09F00BF00BF4B4842
:105BA0000068824503D34A480068824511D34FF00C
:105BB000000B00F00FFF83464648B0F89800401CE9
:105BC00081B24448A0F89810584600F039FF50467A
:105BD000E1E7AAF108073D480088381A1FFA80F962
:105BE0003888A0EB090008381FFA80F800BF00BF12
:105BF000454501DD0020CEE7454501D15046CAE7C5
:105C00000021354800F0EAFE388830490968441818
:105C1000207950BB208809F1080129448EB22F4910
:105C20000968A14204D12949096831442B4A11600D
:105C3000264909688C19002121712080A4F802905E
:105C40003E802188B1F5205F04D021881F4A126868
:105C500011444E801F49B1F89210A8EB0502891A31
:105C60008AB21C49A1F892202AE005F114004045AF
:105C700026D809F10800284486B21448006884191F
:105C800016480068844201D2144804600020207144
:105C900038882080A4F802903E802088B0F5205FEC
:105CA00004D0208809490968084446800948B0F8AA
:105CB0009200A8EB0501401A81B20648A0F89210A4
:105CC000054800F051FF504665E7000084000020C1
:105CD00088000020B8F50020900000208C000020F3
:105CE0002DE9F04104460D4600270DB9BDE8F081CD
:105CF00000BF00BFA5F11C0600F06CFE074600F0D7
:105D0000DBF804EB84010C4800EB41004088401EA6
:105D100081B204EB8402084800EB4200418007484E
:105D200050F824003060054840F82460384600F000
:105D300087FE00BFDAE7000052F60020C44A0020C8
:105D400070B500241CE0002104EB8402224800EB23
:105D50004200418004EB84021F4800EB4200818036
:105D600004EB84021C4800EB4200C1801B4830F861
:105D7000141004EB8402184820F81210601C84B23E
:105D80000C2CE0DB164820F0030500241DE0002069
:105D9000144941F82400002610E0124850F824006D
:105DA0002860104840F824500F4830F8141005F1CE
:105DB0001C00084400F11005701C86B2074830F83A
:105DC0001400B042E9DC601C84B20C2CDFDB00F074
:105DD00033F900F071F870BD52F6002024AA0000DB
:105DE000F74A0020C44A00200CAA00002DE9F04127
:105DF00004460E4617464FF0000800BF0C2C02DB8D
:105E00000020BDE8F08100BF00F0E4FD804600F016
:105E100053F8274850F82450ADB32549286841F875
:105E20002400002028606E60AF6000BF04EB840196
:105E3000204800EB41004088401C81B204EB840202
:105E40001C4800EB4200418004EB8401194800EB40
:105E50004100818804EB8402164800EB4200408830
:105E600081420BDA04EB8401124800EB41004188C7
:105E700004EB84020F4800EB4200818000BF00BFAA
:105E800000BF1C350EE0FFE704EB8401094800EB7E
:105E90004100C088401C81B204EB8402054800EB3D
:105EA0004200C180404600F0CBFD2846A9E7000033
:105EB000C44A002052F6002070B51F4820F00305A8
:105EC000002417E000BF00260DE02146284600F020
:105ED00039F81A4830F8141005F11C00084400F194
:105EE0001005701C86B2164830F81400B042ECDC85
:105EF000601C84B20C2CE5DB0F4820F00305002465
:105F000017E000BF00260DE02146284600F05AF8B1
:105F10000A4830F8141005F11C00084400F110057F
:105F2000701C86B2064830F81400B042ECDC601CED
:105F300084B20C2CE5DB70BDF74A00200CAA0000EF
:105F400024AA0000F0B5A1B006460C461A4830F865
:105F5000141006F11C000F18002529E0785DCD28EB
:105F600024D08022154901A8FAF714FA14A0006879
:105F700000900A2C0ADB0A2094FBF0F03030C0B20B
:105F80008DF80000694601A8FAF728FA0A2094FB68
:105F9000F0F100FB11403030C0B28DF800006946CE
:105FA00001A8FAF71BFA00BF00BF00BF681C85B24A
:105FB000102DD3DB21B0F0BD0CAA00003CAA0000DC
:105FC00030000000F0B5A1B006460C4606F10C0703
:105FD000002529E0785DCD2824D08022144901A82D
:105FE000FAF7D8F913A0006800900A2C0ADB0A20FF
:105FF00094FBF0F03030C0B28DF80000694601A883
:10600000FAF7ECF90A2094FBF0F100FB1140303074
:10601000C0B28DF80000694601A8FAF7DFF900BFA9
:1060200000BF00BF681C85B2102DD3DB21B0F0BDCE
:10603000BCAA0000300000002DE9F041174820F014
:106040000305002425E000BF00261BE005F10C0736
:10605000CD2210213846FAF7AFF9114830F8141064
:1060600005F11C000F18CD2210213846FAF7A4F9CB
:106070000B4830F8141005F11C00084400F110051D
:10608000701C86B2074830F81400B042DEDC601C99
:1060900084B20C2CD7DBBDE8F0810000F74A002069
:1060A0000CAA000024AA00002DE9F04704460D4682
:1060B00016461F46DDE909A9DDF8208000BF00BFB4
:1060C00000206060A060E06084F83500E06120623C
:1060D000C4F828800E48007884F838000C4800780E
:1060E000401C0B490870C4F810903B4632462946C4
:1060F000204600F012F82046D04710B10020BDE83D
:10610000F087044800682060024804602046F6E7F3
:106110009C0000209400002070472DE9F0410646C5
:106120000F4614461D463946304600F017F8214602
:10613000304600F086F82946304600F009F8BDE800
:10614000F0810000014908607047000098000020BD
:1061500009B9002200E00A68C26070472DE9F041E9
:1061600007460C4654B320687968884201D1012063
:1061700000E0002010BB154806680BE03068796825
:10618000884206D1D6F80C80304600F071FE4646B3
:1061900000E0F668002EF1D10D4805680CE055B11D
:1061A000286840B128687968884204D10CB9002079
:1061B00000E020682860ED68002DF0D10CB90020C7
:1061C00000E020687860BDE8F0810000B4000020A5
:1061D000B000002010B5044694F8350000F010001F
:1061E00060B194F8350020F0100084F8350000BF4D
:1061F000206A10B12046216A884700BF10BD10B543
:10620000044694F8350000F01000C8B914F8350FB2
:1062100040F01000207014F8350900F0010040B182
:1062200094F8350000F0200018B1211D2046FEF73B
:1062300007FD00BF206A10B12046216A884700BFD1
:1062400010BD09B9002200E00A688260704710B5ED
:10625000044694F8350000F00100D0B994F83500F8
:1062600040F0010084F8350000BFE06910B120461D
:10627000E169884700BF94F8350000F0100040B194
:1062800094F8350000F0200018B1211D2046FEF7DB
:10629000D7FC10BD2DE9F05F83460F469046BBF159
:1062A000000F09D0BBF1010F08D0BBF1020F07D0DE
:1062B000BBF1030F08D105E038260AE0242608E0E8
:1062C000102606E0002604E000BF00BF0020BDE865
:1062D000F09F00BFB8F1000F78D0B8F1010F72D075
:1062E000B8F1020F70D0B8F1030F6ED1EF2256A1B2
:1062F0000B20FFF77BFD04461CB900F02FFA0020AD
:10630000E5E784F80C800020206006F110002044AE
:10631000C01C20F00300606000BF00BF2781F01C9C
:1063200020F0030040F2EC51081AB84201DD384673
:1063300005E0F01C20F0030040F2EC51081A6081E7
:1063400000BF00BF00BF00BF0120E081A2466089FE
:10635000A7EB000932E04FF488723BA10B20FFF756
:1063600045FD054635B900F0F9F9204600F052F92F
:106370000020ACE785F80C80002068732860CAF81C
:10638000005000BF00BFA5F808901FFA89F040F246
:10639000EC51884202DA1FFA89F001E040F2EC5039
:1063A000688105F11000686000BF00BF00BF00BF3A
:1063B0000120E8816889A9EB0009AA46B9F1000F1C
:1063C000C9DC39E002E020E020E031E006F1130111
:1063D00021F00302F91C21F00301114488B2FFF7F8
:1063E00007FB04460CB9002071E704F110003044AB
:1063F000C01C20F0030060602781678100202060BE
:1064000084F80C8000BF00BF16E000BF4FF4A372F9
:106410000DA10A20FFF7EAFC04460CB9002056E75C
:106420000020606027816781206084F80C8003E091
:1064300000BF00BF00204AE700BF0120E08100202C
:106440006073204643E700002E2E5C2E2E5C5372B4
:10645000635C5573725C4472697665725C55704416
:1064600072697665725C6C7769705C636F72655C8B
:10647000706275662E63000010B5024600BF02B15F
:1064800001B910BD00BF104604E003890C89234404
:10649000038100680368002BF7D100BF00BF00BF75
:1064A00000BF03890C8923440381016000BFE8E732
:1064B0000146002002E0421CD0B209680029FAD14E
:1064C00070472DE9F04105460C460026002700BF25
:1064D00025B11CB128892189884203DA6FF00D00AB
:1064E000BDE8F08100BF00BF6889801B6189C91BBE
:1064F000884204DB6089C01B1FFA80F803E06889CA
:10650000801B1FFA80F86268D1196A6890194246A8
:10651000F9F740FF06EB080086B207EB080087B2E8
:1065200000BF00BF00BF00BF6089B84201DC002788
:1065300024686889B04208D100262D6800BF1DB9C3
:1065400014B16FF00D00CBE700BF54B16089218911
:10655000884206D100BF206810B16FF00500BFE788
:1065600000BF55B168892989884206D100BF2868D3
:1065700010B16FF00500B3E700BF002CB4D10020CC
:10658000AEE72DE9F05F8046894616461D464FF07E
:10659000000B00BFB8F1000F02D10020BDE8F09F52
:1065A00000BF00BFB9F1000F01D10020F6E700BF26
:1065B0004FF0000AB8F1000F02D0B9F1000F01D17D
:1065C0000020EBE7444620E035B16089A84203DCB7
:1065D0006089281A85B217E06089401B87B2B742EC
:1065E00000DD37466268511909EB0A003A46F9F7AF
:1065F000D1FE0BEB07001FFA80FB0AEB07001FFA26
:1066000080FAF01B86B2002524680EB1002CDBD185
:106610005846C3E72DE9F047044624B900BF00BF40
:106620000020BDE8F08700BF00BF00262DE04FF03E
:10663000000900F0CFF9814600BF00BFE089401E8D
:106640001FFA80F8A4F80E80484600F0F9F9B8F176
:10665000000F18D12768257B032D04D121460B207C
:10666000FFF73EFB0BE0012D01D0022D04D12146A6
:106670000A20FFF735FB02E02046FFF72BF9701CDC
:10668000C6B23C4600E0002400BF002CCFD130460B
:10669000C7E7000070B5002500F09CF90546002012
:1066A0000A490870284600F0CBF90948046808E058
:1066B000606F28B1606F02F078FE0020606770BDE7
:1066C000E468002CF4D100BFF9E700009D00002031
:1066D000B400002010B50446FFF7DCFF10BD70B514
:1066E000024600BF00BF01B10AB9002070BD0029F9
:1066F00008DA484284B200BF5089A04201DA012082
:10670000F4E700E08CB2137B55680BB1032B0AD180
:106710005068401A506002F110005668864215D247
:1067200055600120E2E7022B01D0012B0AD100299C
:1067300006DA5089A04203DB5068401A506005E039
:106740000120D3E700BF00BF0120CFE750890844F4
:1067500050811089084410810020C7E770B50025DA
:1067600000F038F905460D48047801200B490870FF
:10677000284600F065F984B900BF00221146084898
:1067800003F01CF940B100F025F90546002003494B
:106790000870284600F054F900BF70BD9D0000202D
:1067A000D56600002DE9F04106460F4600BF00BF48
:1067B00000BF00BF3089B84201DCBDE8F0813089FC
:1067C000A7EB00083D4634460AE06089281A85B2E6
:1067D00000BF00BF208940442081246800BF00BF63
:1067E0006089A842F1DB207B60B96089A84209D0AA
:1067F000A088001B284481B22046FFF7BDF904465B
:1068000000BF00BF658160892081206810B12068C9
:10681000FFF700FF0020206000BFCEE770B5044600
:10682000002544B100F0D6F80546E089401CE0811F
:10683000284600F005F970BD30B500BF00BF00BFAD
:1068400000BF00BF00BF00BF00BF0388194C246811
:106850001919884215D00B799BB9174B1B689942BF
:106860000FD0164B1B688B4201D1144B18600B885C
:106870000380104B1B88C31A0C880E4D2D682C44C6
:10688000638043880B4C24681A19824211D0137913
:106890007BB90A4B1B68834201D1084B1A600388FD
:1068A0001380044B1B88D31A0488024D2D682C4496
:1068B000638030BD84000020880000208C00002010
:1068C0002DE9F04705468A460027D5F8048098F858
:1068D00009900026144804681FE0207C48451AD11E
:1068E00034B1206820B1114920680968884212D16A
:1068F000606980B10E4B2A462146D4E905C0E047C5
:1069000048B10025012736B1E068F060064800680C
:10691000E060054804602646E4680FB9002CDCD12D
:106920003846BDE8F0870000A000002004010020E8
:106930000001002070B504460D4629462046FBF7AD
:10694000FDF970BD704700002DE9F84F81460E46F5
:106950001446D9F800A04CB14FF47A7060434FF45C
:106960007A71B0FBF1F717B9012700E00027FCF7B7
:1069700073FB0446B9B26A46DAF80000FBF788FDFB
:1069800080463EB11248804502D10020306001E0CF
:10699000C6F800809DF800000A2802D14FF0FF34AD
:1069A00013E000BF00BFFCF757FB0546A54201D925
:1069B0002D1B02E0C4F1FF3005444FF47A706843A8
:1069C0004FF47A71B0FBF1F0441C2046BDE8F88F1B
:1069D0001401002010B5F9F765FC10BDF8B50746A5
:1069E0000C464CB14FF47A7060434FF47A71B0FBAF
:1069F000F1F616B9012600E00026FCF72DFB04464F
:106A0000B1B26A463868FBF7B9FE9DF800000A2863
:106A100002D14FF0FF3411E0FCF71EFB0546A54202
:106A200001D32D1B02E0C4F1FF3005444FF47A700E
:106A300068434FF47A71B0FBF1F0441C2046F8BD76
:106A400010B504462046F9F731FC10BD08B56B4679
:106A5000542214210248FBF753FC0249086008BD88
:106A6000B4F700200C01002038B504460D46142D63
:106A700000DD142569460E480068FBF77FFC2060A6
:106A80009DF8000080B9A9B22268101DFBF7B0FC88
:106A9000216808602068006808B1002038BD2146E0
:106AA00003480068FBF789FC4FF0FF30F6E7000071
:106AB0000C01002070B504460D4605B9044D00BF19
:106AC000216808682946FBF775FD0028F8D170BDDC
:106AD0001401002070B505460E4606B9064E296819
:106AE00008683146FBF766FD04460CB9002070BD0E
:106AF0004FF0FF30FBE7000014010020F0B585B037
:106B00000446256814216846F9F75DFC6946286843
:106B1000FBF789FD0646022E07DABDF80400BDF832
:106B20000610884201DA012000E0002007463846BE
:106B300005B0F0BD38B504460D462846FBF7F4FD18
:106B40002060206810B94FF0FF3038BD6A4603A1BD
:106B50002068FBF70DFB0020F7E700004C57495079
:106B60002053656D0000000010B504462068FBF757
:106B70007DFE10BD2DE9F04385B080460D461646DA
:106B80001F460C9C4FF0000900BF00BF10A14046FB
:106B9000F9F730FCB0B9F9F785FB814603200021F5
:106BA0004FF400620E4BCDE90132CDE90310A0B2E3
:106BB000E3B20C4A00902846FBF7D4FE4846F9F7AA
:106BC00075FB00E00024E0B205B0BDE8F0830000F2
:106BD00074637069705F74687265616400000000BE
:106BE00044FE0020401E01202DE9F04106460F46DC
:106BF000904640F20F1224A10920FFF7F7F804464F
:106C00001CB900BF00BFBDE8F08100202060A76074
:106C1000C4F80C8066602948006810B927480460F1
:106C2000F1E7264800684068B0420CD92348006864
:106C30004068801B2149096848602048006820603E
:106C40001E4804601DE01D48056817E0606869681B
:106C5000401A6060286820B12868406861688842EE
:106C60000BD9286828B1286840686168401A2968EB
:106C70004860286820602C6002E02D68002DE5D176
:106C800000BF00BFBFE700002E2E5C2E2E5C5372AB
:106C9000635C5573725C4472697665725C557044CE
:106CA00072697665725C6C7769705C636F72655C43
:106CB00074696D6572732E6300000000E8000020A7
:106CC00010B50022024941F28830FFF78DFF10BD58
:106CD000A54400002DE9F0478046894600BF2248C0
:106CE000006830B9002249464046FFF72DFE0546B0
:106CF00037E01D480068406840B11B4800684946BD
:106D000042684046FFF720FE054601E04FF0FF35A0
:106D1000681CA8B914480468134920680860A6686C
:106D2000E76821460920FEF7DBFF46B100210F4846
:106D3000FFF754FE3846B0470C48FFF715FFCEE783
:106D4000094800684068A84207D9074800684068B9
:106D5000401B05490968486003E0002002490968B2
:106D60004860BDE8F0870000E800002080000020B7
:106D70002DE9F04106460F461448006808B9BDE801
:106D8000F0811248046800251BE0A068B04216D1CB
:106D9000E068B84213D11DB90C492068086001E0D1
:106DA00020682860206828B120684068616808442D
:106DB0002168486021460920FEF792FFDFE725465B
:106DC0002468002CE1D100BFD9E70000E8000020D2
:106DD0002DE9FC4704460E4600BF00BF207E0A286E
:106DE00008D121461F4801F057F921460220FEF73D
:106DF00077FF34E0276DD4F82880D4F88C50D4F88D
:106E0000109000BF2146184801F046F901201749AB
:106E1000087000BF206F10B1206F02F0C6FAE06E5C
:106E200010B1E06E02F0C1FA606F10B1606F02F055
:106E3000BCFA4EB1A08B618B231D2246CDE9001018
:106E40004146384602F02EFA21460220FEF748FF5E
:106E500000BF1DB16FF009014846A84700BFBDE85B
:106E6000FC870000B8000020B4000020C000002013
:106E700010B5044601212046FFF7AAFF10BD00000F
:106E800070B5064640F2035239A10220FEF7AEFF6C
:106E90000446002C25D100F0DDFD40F2095234A15A
:106EA0000220FEF7A3FF044694B9304600F0A8FD87
:106EB00040F20F522EA10220FEF798FF04463CB18B
:106EC0003748B0F8B400401E81B23548A0F8B4107D
:106ED0003CB13348B0F8B400401E81B23048A0F84D
:106EE000B410002C41D0A0212046F9F76CFA1834D8
:106EF000667041F2D060A4F84E000020A4F8500063
:106F000042F23820A082E082002004F80F0CFF201B
:106F100004F80E0C4FF40670E0830620A0850020D4
:106F2000208506206085C01FA0830120A08600F078
:106F300051FE05462564A56325636564194800680C
:106F4000E0601948007860720020E0711748A06680
:106F500040F6B830A0674FF4FA60E0670620C4F846
:106F60008000002084F88600183C204670BD000098
:106F70002E2E5C2E2E5C5372635C5573725C4472D1
:106F8000697665725C55704472697665725C6C777F
:106F900069705C636F72655C7463702E63000000DF
:106FA000B8F50020A8000020C20000202D910000AC
:106FB00010B50446207E012803D0A07F40F01000C9
:106FC000A0770121204600F001F810BD7CB50446F1
:106FD0000E46002E5BD0207E042802D0207E07289B
:106FE00055D1A06F20B9A08D42F2382188424ED0F1
:106FF00000BF00BFA08B618BCDE90010231D22468E
:10700000A16A206D02F04EF9204601F021F800BF80
:1070100000BF5A480068A04205D158480068C068BF
:107020005649086018E055480068554908600EE068
:1070300053480068C068A04204D15149E06809681B
:10704000C86008E04E480068C0684D4908604C4878
:1070500000680028ECD100BF0020E06000BF0120E4
:107060004849087000BF207E04280AD10A202076F3
:1070700000BF45480068E0604348046002F096FBAA
:1070800003E021460220FEF72BFE00207CBD207E7F
:10709000082868D2DFE800F004343F4F5767675F85
:1070A0000025608B30B300BF38480068A04205D18E
:1070B00036480068C0683549086018E03348006801
:1070C0002F4908600EE02E480068C068A04204D135
:1070D0002B49E0680968C86008E029480068C06872
:1070E00027490860264800680028ECD100BF00202E
:1070F000E06000BF21460220FEF7F2FD002435E0EB
:1071000000252146224800F0C7FF21460320FEF754
:10711000E7FD00242AE0002500BF2146174800F0C3
:10712000BBFF01201749087000BF21460220FEF76F
:10713000D7FD00241AE0204602F06AF905460DB991
:107140000520207612E0204602F062F905460DB9CE
:10715000052020760AE0204602F05AF905460DB9CE
:107160000920207602E00025002400BF00BF1CB1EA
:1071700015B9204600F084FD284687E7B4000020BA
:10718000BC000020C0000020B8000020AC0000209F
:10719000B00000202DE9F05F07460E4691469A4662
:1071A000DDF8288008F0010008B1042000E000208C
:1071B00008F0020109B10C2100E000214518A422C9
:1071C00024A10420FEF712FE041E05D13046FFF76D
:1071D00021FA0020BDE8F09F84F80A80002020609A
:1071E00066603089401B208114213046FFF777FA12
:1071F00060B12548B0F88C00401C81B22248A0F84C
:107200008C10204602F0C4F80020E3E76068406874
:10721000E060788BFEF7B3FAE1680880B88BFEF780
:10722000AEFAE16848805046FEF79CFAE168486093
:10723000AB46E91705EB91718910491D49EA013107
:1072400088B2FEF79CFAE16888810020E1684882F4
:107250002046BFE72E2E5C2E2E5C5372635C557366
:10726000725C4472697665725C55704472697665C9
:10727000725C6C7769705C636F72655C7463705F7D
:107280006F75742E63000000B8F500202DE9F04101
:1072900005460E463046FEF741F9044654B1A08D2E
:1072A00040B1A08D283887B2BD4201DA284600E0FF
:1072B000384605462846BDE8F08100002DE9F84330
:1072C00004460D460027B84600BF00BFB4F868006A
:1072D000102805DAB4F868004FF6FC7188420FD91F
:1072E0004A48B0F88400401C81B24848A0F8841095
:1072F000A07F40F08000A0774FF0FF30BDE8F8831A
:1073000005F0020000B1012707F0010008B10420D8
:1073100000E0002007F0020109B10C2100E000218B
:1073200000EB0108B4F8660050B93848B0F88400A2
:10733000401C81B23548A0F884104FF0FF30DDE7E3
:10734000002241461046FEF7A5FFB0F100090ED11C
:10735000A07F40F08000A0772C48B0F88400401C4B
:1073600081B22A48A0F884104FF0FF30C6E700BF72
:1073700000BF00972A4649462046E36DFFF70AFF03
:10738000061E0DD1A07F40F08000A0771F48B0F806
:107390008400401C81B21D48A0F88410701EADE727
:1073A00000BF00BF00BF00BFE06E08B9E66607E09F
:1073B000E06E00E0006801680029FBD1066000BFB4
:1073C0000020A4F86A0005F0020010B905F00100E1
:1073D00038B1E06D401CE065B4F86600401EA4F8CA
:1073E000660005F0010018B1A07F40F02000A077F2
:1073F0007068FFF75DF834F8681F0844208034F89F
:10740000680908B100BF00BF002077E7B8F5002089
:1074100070B51B480078401C1949087000BF194816
:10742000046829E094F8210015490978884223D09E
:107430001348007884F82100A07F00F0010060B1BB
:1074400000BFA07F40F00200A07700BF204600F000
:1074500017FCA07F20F00300A077E568A06F48B17B
:10746000002009490870204601F026F906480078F6
:1074700000B1D4E72C4600BF002CD3D170BD000072
:10748000C2000020B4000020C000002070470000AF
:107490002DE9FC4706468A46FB48B0F87A00401CB6
:1074A00081B2F948A0F87A10F84970680860F74886
:1074B00071680068007800F00F0001EB8000F4496B
:1074C0000860F248006800780007800E41423046AC
:1074D000FFF705F910B93089142808D2EA48B0F846
:1074E0008200401C81B2E848A0F882103BE2E949E2
:1074F00008685146FDF75DFE28B9E648007800F0BF
:10750000F000E02808D1E048B0F88800401C81B2C3
:10751000DD48A0F8881026E2DD4909688889FEF771
:107520004EF94FEA20394FEA890041423046FFF7D1
:10753000D6F840B1D448B0F88200401C81B2D2489D
:10754000A0F882100FE2D24909680888FEF737F9DF
:10755000CF4909680880CE4909684888FEF72FF9A5
:10756000CB4909684880CA4909684868FEF721F98B
:10757000C74909684860C8490860C54909688868FA
:10758000FEF717F9C24909688860C4490860C04914
:107590000968C889FEF713F9BD490968C881BC4963
:1075A00009688889FEF70BF900F03F00BC490870B4
:1075B0003089097801F0030109B1012100E00021BF
:1075C0000844B84908800027B74804682AE000BF8B
:1075D00000BF00BF00BF00BF00BFA08BAC4909685F
:1075E000098888421CD1608BA9490968498888426A
:1075F00016D1AE4960680968884211D1A549206852
:10760000096888420CD100BF00BF37B1E068F8605C
:10761000A5480068E060A448046000BF00BF03E024
:107620002746E468002CD2D100BF002C4DD1A048E1
:10763000046820E000BF00BFA08B95490968098855
:10764000884217D1608B924909684988884211D1D4
:1076500096496068096888420CD18E49206809689B
:10766000884207D1204602F0BDF83046FEF7D2FF2F
:10767000BDE8FC87E468002CDCD100278D48056854
:1076800010E0688B824909684988884208D181499D
:1076900028680968884202D00DB1286800B903E063
:1076A0002F46ED68002DECD100BF75B137B1E86809
:1076B000F86080480068E8607E480560284600F071
:1076C000E7F93046FEF7A6FFD2E7002C7ED0002077
:1076D0007949086030890881084646606C4800682E
:1076E000C860002075490860754908706C480078CA
:1076F00000F0080018B1707B40F001007073A06FBB
:1077000098B1204600F0D8FF0A3028B1A06F60B1D0
:1077100064480088002808DD5B48B0F87E00401C03
:1077200081B25948A0F87E10DDE06648046020462A
:1077300000F0FCFC804608F10A00002817D06048E1
:10774000007800F0080098B100BFD4F88C0028B190
:107750006FF00A01D4F88C202069904700BF2146C1
:10776000514800F099FC21460220FEF7B9FAB9E031
:107770005348007800F01000B8B1A07F00F010006E
:1077800050B900BFD4F88C0028B16FF00B01D4F8C9
:107790008C202069904700BF2146434800F07CFCC4
:1077A00021460220FEF79CFA9CE04FF00008B4F856
:1077B0006400002812DD00BFE06F40B1B4F864201F
:1077C0002146E36F20699847804602E09BE04FF036
:1077D000000800BF08F10A0000B984E037480068DB
:1077E00070B300BF00BFA07F00F0100038B1334875
:1077F0000068FEF70FFF2046FFF73AFB73E000BF7B
:10780000D4F8800048B100232C49D4F880C0206906
:107810000A682146E047804607E0002327482146C2
:107820000268184601F082FC804600BF08F10A0099
:1078300000B958E0B8F1000F02D020480068A067F6
:107840001F48007800F02000E8B1A06F30B1A06FB1
:10785000407B40F02000A16F48733DE0A08D42F2D4
:107860003821884202D0A08D401CA08500BFD4F8EA
:10787000800048B300231A462146D4F880C020690E
:10788000E047804623E027E0B8F50020CC00002048
:10789000C800002004010020D0000020D4000020F7
:1078A000D8000020DA000020B400002000010020F1
:1078B000B8000020B0000020DCF60020E00000202E
:1078C000DC000020E4000020FFE74FF0000800BFCC
:1078D00008F10A0000B906E00020294908602046A6
:1078E00000F0CEF900BF0020254908602549086056
:1078F00025484068A0B324494868FEF78BFE002065
:10790000214948602CE0214909688889FDF757FF23
:1079100000F0040008BB1E48B0F88800401C81B28B
:107920001B48A0F88810B0F87E00401C81B21848AF
:10793000A0F87E1015480068008814490968498835
:10794000CDE9001013480068134A12888118134BC0
:10795000134A1448006801F0A5FC3046FEF75AFEB1
:1079600000BF00BF84E60A48B0F87E00401C81B228
:107970000748A0F87E103046FEF74CFE00BF77E6C1
:10798000E4000020E0000020DCF60020C800002019
:10799000B8F50020D0000020DA000020000100200F
:1079A00004010020D40000202DE9FC410446216D93
:1079B000481EFDF7D7FE07463B46002211462046EB
:1079C00000F03EFA05460DB9BDE8FC816E680B4833
:1079D000B0F87800401C0949A1F878000620002181
:1079E000CDE90010A37A221D21462846FDF70CFDA3
:1079F0002846FEF70FFE00BFE6E70000B8F50020BE
:107A00002DE9F04106464FF07F08002700250F487A
:107A1000046813E0607EB0420FDC607E40450CDC01
:107A20000B49606A0968081AB84206D30849606AB7
:107A300009680F1A254694F81980E468002CE9D1EA
:107A400015B12846FFF714FABDE8F081B400002014
:107A5000A800002070B5002600250B4804680BE044
:107A60000A49606A0968081AB04204D30749606A83
:107A700009680E1A2546E468002CF1D115B1284694
:107A8000FFF7F6F970BD0000B8000020A800002044
:107A90007CB505464548007800F0040008B1002098
:107AA0007CBD4248007800F0100098B14048006862
:107AB00000883F4909684988CDE900103D480068C1
:107AC0003D4A128881183D4B3D4A3E48006801F00E
:107AD000E9FB69E03548007800F00200002863D037
:107AE000687EFFF7CDF9044654B93748B0F88400F2
:107AF000401C81B23448A0F884104FF0FF30CFE72B
:107B00002F4800682060688B60832C4800686060A4
:107B1000274800680088A083032020762548006855
:107B2000401CA062A06A206321480068C089A4F8B4
:107B300060001F480068C089A4F86200B4F86000C3
:107B4000A4F84E001B480068401E6065286920614B
:107B500068696061287A00F08C00207200BF00BF65
:107B60001A480068E0601948046001F01FFE00BF79
:107B700001201749087000BF204600F00DFAE08E82
:107B8000211DFFF783FBE08612212046FFF796FBBD
:107B900006462EB100212046FFF71AF930467FE74E
:107BA000204600F06DF87BE7002079E7D800002040
:107BB000C8000020D0000020DA00002000010020D2
:107BC00004010020D4000020B8F50020B4000020FB
:107BD000C0000020044800680449096808440249BC
:107BE0000860084600687047C4000020A800002014
:107BF00070B505460C46E9688889FDF7E0FD00F0A0
:107C0000010020B1204601F0D0FB002433E013E056
:107C1000E1688889FDF7D3FD00F0010038B101204B
:107C2000FDF7ADFDE96889890843E9688881264642
:107C30002468304601F0ACFB4CB1E0684068218913
:107C4000084429890D4A12681144081AE0D594B1F4
:107C500028890A4909680844E1684968401A0028E7
:107C600009DDE068808805490988401A288129894A
:107C70006868FEF797FD2C6070BD0000D000002002
:107C80002DE9F047044600BF00BF6C480068A042E1
:107C900002D10020BDE8F087B4F86000B4F84C10C1
:107CA000884202DAB4F8600001E0B4F84C00814682
:107CB000E56EA07F00F0020070B14DB1E968486840
:107CC000FDF777FDA16C401A29890844484503D97E
:107CD000204601F076FBDDE7266F26B100E036682E
:107CE00030680028FBD191E000BFE9688889FDF782
:107CF00066FD00BF206FA0B1A07F00F0440080B9F6
:107D0000E06E38B1E06E006858B9E06E0089E18E2F
:107D1000884206DAB4F8660018B1B4F86800102892
:107D200001DB012000E0002020B9A07F00F0A000CE
:107D300000B977E02868E066207E02280BD010208A
:107D4000FDF71DFDE96889890843E9688881A07FFE
:107D500020F00300A0772146284600F0ADF8E9683E
:107D60004868FDF726FD0746E9688889FDF727FD85
:107D700000F0030008B1012000E000202989084438
:107D800007EB0008206DB0EB080001D5C4F8508067
:107D9000E9688889FDF713FD00F0030008B10120B0
:107DA00000E000202989084400282BDD00202860FD
:107DB000206F10B925672E4627E0E9684868FDF76F
:107DC000F8FC0746F1684868FDF7F3FC381A16D549
:107DD00004F1700700E03F68386860B13968C9682D
:107DE0004868FDF7E6FC8246E9684868FDF7E1FC73
:107DF000BAEB0000EFD4386828603D6005E03560DC
:107E0000366802E0284601F0C3FAE56E55B1E9682C
:107E10004868FDF7CEFCA16C401A29890844484502
:107E20007FF662AF00BFE06E10B90020A4F86A00D0
:107E3000A07F20F08000A07700202BE7E400002046
:107E40002DE9F04705460E469046994606F1140086
:107E5000404481B200220120FEF71CFA074647B3D6
:107E600000BF00BF7C68688BFDF789FC2080A88B71
:107E7000FDF785FC6080C4F80490A86AFDF772FCE9
:107E8000A060B246F11706EB91718910491D1022CE
:107E900042EA013188B2FDF772FCA081E88DFDF75E
:107EA0006EFCE081002020826082E98DA86A08448F
:107EB00028633846BDE8F0872DE9FC4705460C46A7
:107EC000A06AFDF74FFCE9688860E08DFDF757FC7C
:107ED000E968C881E18DA06A08442063E86800F180
:107EE0001408A87A00F0010070B1211D40F2B450CE
:107EF000FFF7CCF9814649F00170FDF733FCC8F873
:107F0000000008F1040800BFB4F93400401C08B9AF
:107F10000020A0860CB1206840B9201DFDF7FEFAB4
:107F200006460EB9BDE8FC8770682060A06B38B9C2
:107F300017480068A063E9684868FDF73AFCE06309
:107F4000A88969688988401A87B268684089C01B17
:107F50006968488168680089C01B69680881696828
:107F6000E86848600020E96808820A48B0F87800AC
:107F7000401C0849A1F878000621607ACDE900018B
:107F8000A37A221D21466868FDF73EFA00BFC9E7C3
:107F9000A8000020B8F500202DE9F04780462B48C6
:107FA000006800F11405294909688889FDF707FC74
:107FB0000521B1EB203F46DA244909688889FDF79D
:107FC000FEFB0521C1EB20304FF6FF7101EA800670
:107FD000002436E015F80490B9F1000F06D0B9F18D
:107FE000010F05D0B9F1020F21D104E0BDE8F087FF
:107FF000601C84B224E0601C285C042802D1201D8F
:10800000B04200DDF2E7E01C295CA01C285C41EADC
:10801000002740F2B450874200DC17B940F2B45058
:1080200000E03846A8F83600201D84B208E0601C45
:10803000285C00B9DAE7601C285C204484B200BFE9
:1080400000BFB442C6DB00BFD0E70000C80000207C
:1080500010B50446207EF0B1207E0A281BD0207E79
:10806000012818D0A06F20B1A06FFEF7D3FA00202E
:10807000A067606F01F099F900206067401EA0863C
:10808000E06E01F092F9206F01F08FF90020E066B8
:108090002067A4F86A0010BD70B505460C4600BF05
:1080A0002868A04203D12868C068286017E01E49EC
:1080B000286808600EE01C480068C068A04204D12F
:1080C0001949E0680968C86008E017480068C06896
:1080D00015490860144800680028ECD100BF002052
:1080E000E06000BF2046FFF7B3FF207E0A280DD0D6
:1080F000207E01280AD0A07F00F0010030B1A07FCF
:1081000040F00200A0772046FFF7BAFD207E01284C
:1081100005D000BF00BF00BF00BF00BF00BF0020F0
:10812000207600BF00BF70BDBC0000202DE9FC41DF
:1081300004464FF000080026FE48007800F00400D6
:1081400070B3207E022807D1FB49206D0968884260
:1081500011D14FF001080EE0F849A06A0968081A29
:1081600009D4A18DA06A0844F4490968081A0028B6
:1081700001DC4FF00108B8F1000F0FD000BF00BFC5
:10818000EF48007840F00800ED490870A07F20F02B
:108190000100A0776FF00A00BDE8FC810020FBE73A
:1081A000E448007800F0020068B1207E02280AD07E
:1081B000207E032807D000BFA07F40F00200A077F8
:1081C00000BF0020E8E7A07F00F0100010B9DD48F4
:1081D00000686062002084F89E002046FFF7DCFE05
:1081E000207E801E082873D2DFE800F0049BF0EFA9
:1081F000EEEDECEBCF48007800F01000002877D0CF
:10820000CC48007800F00200002871D0216FC968C6
:108210004868FDF7CEFA401CC7490968884267D113
:108220002834E08F401CE087C4480068401C206070
:108230002068A060C04800682062C3480068C08908
:108240002087C1480068C0896087BC480068401E1C
:10825000E062042004F8100CE089283C211DFFF79F
:1082600015F8E086E08E00EB80004FF6FF7101EA22
:108270004000A4F84E00B4F84C00012802D1E08E72
:10828000400000E0E08EA4F84C0000BF00BFB4F84E
:108290006800401EA4F86800256F286820672846FB
:1082A00001F076F8206F18B94FF0FF30A08603E098
:1082B0000020A08684F8460000BFD4F8840048B1AE
:1082C00000222146D4F8843020699847064602E00F
:1082D000E0E10DE0002600BF06F10A0010B96FF0E2
:1082E000090059E700BFA07F40F00200A07717E027
:1082F0009048007800F0100090B193480068008822
:10830000914909684988CDE900108C4800688F4A76
:10831000128881188E4B8F4A8748006800F0C2FF90
:10832000B9E18448007800F01000002863D0A06C08
:10833000401C81490968081A49D47F49206D0968A1
:10834000081A002843DC0420207600BF00BF00BFCD
:10835000606930B100222146D4E9040398470646FB
:1083600001E06FF00D0600BF46B106F10A0010B142
:108370002046FEF77DFD6FF009000DE7B4F84C7064
:10838000204600F0E1F9B4F8640020B1B4F86400CC
:10839000401EA4F86400012F02D1E08E400000E0EE
:1083A000E08EA4F84C006648007800F0200038B158
:1083B00000BFA07F40F00200A07700BF072020761A
:1083C00027E053E108E125E0A1E035E023E05E4845
:1083D000006800885C4909684988CDE90010574861
:1083E00000685A4A12888118594B5A4A5248006804
:1083F00000F058FF0DE04F48007800F0020040B157
:10840000A06A401E4D490968884202D1204600F00A
:10841000C7FE40E100BF204600F096F948480078CA
:1084200000F0200038B100BFA07F40F00200A0772C
:1084300000BF072020762EE1204600F085F9404855
:10844000007800F02000E8B33A48007800F010000F
:10845000C8B33949206D0968884242D100BFA07F66
:1084600040F00200A07700BF2046FFF7F1FD00BFFB
:1084700000BF39480068A04205D137480068C0688D
:108480003549086018E034480068344908600EE057
:1084900032480068C068A04204D13049E0680968E9
:1084A000C86008E02D480068C0682C4908602B4867
:1084B00000680028ECD100BF0020E06000BF012070
:1084C000274901E016E00CE0087000BF0A20207682
:1084D00000BF24480068E0602248046001F066F9AB
:1084E00014E000BFA07F40F00200A07700BF08208A
:1084F00020760BE00F48007800F0100030B10E49F4
:10850000206D0968884201D106202076C3E020460C
:1085100000F01AF90A48007800F0200078B300BF94
:10852000A07F40F00200A07700BF2046FFF790FD3B
:1085300000BF19E0D8000020D4000020D0000020A7
:10854000DC000020A8000020C8000020DA00002085
:108550000001002004010020B4000020BC00002025
:10856000C0000020B800002000BF4C480068A042B6
:1085700006D14A480068C0684849086019E02AE006
:1085800046480068464908600EE045480068C068F3
:10859000A04204D14249E0680968C86008E0404848
:1085A0000068C0683E4908603D4800680028ECD17A
:1085B00000BF0020E06000BF01203A49087000BF02
:1085C0000A20207600BF38480068E0603648046022
:1085D00001F0ECF800BF5EE0204600F0B5F833484B
:1085E000007800F01000E0B33149206D096888423E
:1085F0003BD12046FFF72CFD00BF00BF2748006895
:10860000A04205D125480068C0682449086018E0E8
:1086100022480068224908600EE021480068C068CE
:10862000A04204D11E49E0680968C86008E01C48FF
:108630000068C0681A490860194800680028ECD131
:1086400000BF0020E06000BF01201649087000BF95
:108650000A20207600BF14480068E06012480460D9
:1086600000E002E001F0A2F800BF14E0204600F0B4
:108670006BF80E48007800F0100050B10C49206DE6
:108680000968884205D10B48007840F0100009497C
:10869000087000E000BF00BF00207DE5B4000020AE
:1086A000BC000020C0000020B8000020D80000203E
:1086B000D4000020DC0000202DE9F0410446A06F2A
:1086C000477BA66F0020A06700BFD4F8800040B1B0
:1086D000002332462146D4F880C02069E047054691
:1086E00006E0002332462146184600F01FFD0546ED
:1086F00000BF05BB07F0200020B3A08D42F2382157
:10870000884202D0A08D401CA08500BFD4F8800014
:1087100040B100231A462146D4F880C02069E047C2
:10872000054600E0002500BF05F10A0050B96FF0D2
:108730000900BDE8F08105F10A0010B96FF00900E9
:10874000F7E7A6670020F4E72DE9FE4F0446002076
:10875000009000BF00BFFE48007800F01000002825
:108760007ED0B4F86000A16D08440290F949606DB4
:108770000968401A15D4F749606D0968884204D128
:10878000F549A06D0968401A0BD4F349A06D09683A
:10879000884231D1F1480068C089B4F8601088423D
:1087A0002ADDEE480068C089A4F86000B4F86200D1
:1087B000EA490968C989884204DAE8480068C0893A
:1087C000A4F86200E34800686065E3480068A065BB
:1087D000B4F8600048B994F89D0068B9002084F8A6
:1087E0009C00012084F89D0006E094F89D0000287C
:1087F00002DD002084F89D00D749A06C0968081AA2
:10880000002848DC0020A4F86400D548008840BB5C
:10881000B4F86010A06D01440298814235D1B4F9DA
:108820003400002831DBCC49A06C096888422CD187
:108830000120009094F84700401CC0B294F8471003
:10884000884204DD94F84700401C84F8470094F8FF
:108850004700032812DDB4F84C00E18E084401E023
:108860004AE10AE080B2B4F84C1088420DDDB4F859
:108870004C00E18E0844A4F84C0006E094F8470050
:10888000032802D1204600F0B8FC0098002801D14E
:1088900084F84700ADE0A06C401CAF490968081A95
:1088A0007ED4AD49206D0968081A002878DCA07FC5
:1088B00000F0040038B1A07F20F00400A077B4F8E5
:1088C0004E00A4F84C0000202834A077608BB4F947
:1088D000181000EBE10000B2A083208C9E490988AB
:1088E000081AA087E08FA18F0844E0870020E07776
:1088F00099480068206214F8100C283C042824DBF6
:10890000B4F84C00B4F84E1088420FDAB4F84C00BA
:10891000E18E084480B2B4F84C10884215DDB4F8FA
:108920004C00E18E0844A4F84C000EE034F8361FE9
:108930004943E28A91FBF2F1114488B2E18A363C64
:10894000814201DAA4F84C0000BF26E0256F206FB9
:108950000068206700BF6868FDF7AAFD00BFB4F893
:10896000640058B1E9688889FCF729FF00F001002C
:1089700020B1B4F86400401EA4F864006868FDF7F4
:1089800097FD34F8681F081A2080284600F000FD83
:1089900034F8680908B100BF00BF206FD8B100E00B
:1089A00024E0216FC9684868FCF703FF8346216F04
:1089B000C9688889FCF703FF00F0030008B10120B3
:1089C00000E00020216F0989084458446249096881
:1089D000401A0028BADD206F18B94FF0FF30A0868A
:1089E00001E00020A0860020E07702E00020A4F84B
:1089F00064002BE0E56EE06E0068E066E06E10B9A2
:108A00000020A4F86A0000BF6868FDF751FD00BFB0
:108A1000B4F8640058B1E9688889FCF7D0FE00F02A
:108A2000010020B1B4F86400401EA4F86400686836
:108A3000FDF73EFD34F8681F081A2080284600F034
:108A4000A7FC34F8680908B100BF00BFE06EF0B1C0
:108A5000E16EC9684868FCF7ACFE8346E16EC96800
:108A60008889FCF7ACFE00F0030008B1012000E0AB
:108A70000020E16E09890844584437490968081AFA
:108A800005D43549206D0968081A0028B2DDA06BAD
:108A900090B33149E06B0968401A2DD534F8380F8E
:108AA00030490988081A0FFA80FAB4F90800AAEBCD
:108AB000E0000FFA80FA2089504400B22081383C4F
:108AC000BAF1000F03DACAF100000FFA80FA383465
:108AD000B4F90A00AAEBA0000FFA80FA60895044AA
:108AE00000B260816089B4F9081000EBE10000B2C7
:108AF000A081002044F838091948008800286EDD5C
:108B0000207E07286BDA1348A16A0068401C081A07
:108B100066D41048A16A0068114A12881044401EA9
:108B2000081A00285CDC0B49A06A0968A0EB01095F
:108B30000D48D0F8048000BF00BF00BF00BF4068F0
:108B40004089484531DA00BF00BF074840680DE062
:108B5000D8000020D0000020D4000020C800002051
:108B6000DA000020A8000020DCF600200089A0EB3D
:108B7000090080B201900BE0B8F80A00A9EB0009E7
:108B80000198A8F808000020A8F80A00D8F800808A
:108B9000B8F80A004845EFDBC9F1000001B24046D1
:108BA000FDF79DFD58B100BF09E0F8494868C9F1DB
:108BB000000109B2FDF793FD08B100BF00BFF34803
:108BC0000089218DF24A1288891A401AEF490881DA
:108BD000EF49A06A0860ED49C96848600BE089E286
:108BE000EB49A06A0968081A05D500BFA07F40F0CC
:108BF0000200A07700BFE649A06A0968081A6FD48E
:108C0000A18DA06A0844401EE1490968081A00289D
:108C100066DCDF49A06A096888426FD1DB49C96810
:108C20008889FCF7CCFD00F0030008B1012000E0CA
:108C30000020D64909890844D6490880A08D0988B2
:108C4000884241DAD149C9688889FCF7B8FD00F04B
:108C5000010098B1CD49C9688889FCF7B0FD00F0E2
:108C60003E0B5846FCF78BFDC849C96889894CF210
:108C7000FF0211400843C549C9688881A08DC349D6
:108C80000881C9688889FCF79AFD00F0020020B1CC
:108C9000BE480089401EBD490881BC4A1189506800
:108CA000FDF780FDB949C9688889FCF788FD00F0A7
:108CB000030008B1012000E00020B44909890844FC
:108CC000B449088000BF00BF606F002815D0AF49CD
:108CD000C9688889FCF773FD00F0010078B109E0EC
:108CE00004E2D4F874B0606F00686067584600F022
:108CF0004FFB00BF606F0028F3D172E00DE1656F9C
:108D00002DE0E9688889FCF75AFD00F0010008B3FE
:108D10009E49C9688889FCF752FD00F00200C8B975
:108D20000120FCF72CFD9949C968898908439749B6
:108D3000C96888819549C9688889FCF740FD00F0B9
:108D4000030008B1012000E000209049098908448F
:108D5000904908802F462D68384600F019FB55B120
:108D6000E86840682989014489480068894A12886E
:108D70001044401AC5D59DB38548006885490988C7
:108D80000844E9684968401A002829DDE8688088B5
:108D90007F490988401A7D490881C9688889FCF79C
:108DA0000EFD00F0020020B178480089401E77498E
:108DB0000881764A11895068FDF7F4FC7349C96847
:108DC0008889FCF7FCFC00F0030008B1012000E0FA
:108DD00000206E49098908446E49088000BF00BF21
:108DE00065676B4800686B4909880844A06200BF4A
:108DF00000BFA08D67490988401AA085204600F071
:108E000059FD624840680089002806DD5F484068D7
:108E10006149086000205D4948605C49C9688889EB
:108E2000FCF7CDFC00F0010028B15C48007840F070
:108E300020005A49087055E0666F606FC06840684E
:108E400053490860F1688889FCF7B9FC00F0030019
:108E500008B1012000E0002031890844A16A0844DB
:108E6000A06200BFF1688889FCF7A9FC00BFF16827
:108E70008889FCF7A4FC00F0030008B1012000E0A1
:108E8000002031890844A18D081AA085204600F0F1
:108E900011FD7068008900280DDD3F48006828B189
:108EA0003D4871680068FDF7E7FA02E03A497068EA
:108EB000086000207060F1688889FCF780FC00F091
:108EC000010050B13548007840F020003349087067
:108ED000207E042801D10720207630686067304664
:108EE00000F056FA606F28B1606FC0684068A16AF0
:108EF0008842A1D000BFA07F00F0010040B1A07F58
:108F000020F00100A077A07F40F00200A07703E0EE
:108F1000A07F40F00100A07700E1204600F051FA68
:108F2000606F20B9194800F005FA6067F6E0002785
:108F3000656FD7E0E868406815490968884213D131
:108F400012480089298988420DDD104800F0F2F9A5
:108F500006463EB10FB13E6000E0666729463046E6
:108F6000FEF746FEC1E0C0E0D7B9E86840680849AE
:108F70000968081A41D5054800F0DCF9064626B113
:108F8000666729463046FEF733FEAEE0DCF6002089
:108F9000D0000020DA000020E0000020DC000020EB
:108FA000F8684068401C5E490968081A25D4E868DA
:108FB0004068401E5A490968081A00281DDC5948B3
:108FC00000F0B8F90646BEB1F8684068398908442F
:108FD00053490968401A002809DDF868808850491B
:108FE0000988081A388139897868FDF7DBFB3E600B
:108FF00029463046FEF7FCFD77E02868E8BBE868C4
:10900000406847490968081A002869DDE9688889C5
:10901000FCF7D5FB00F0010000B166E0414800F02C
:1090200089F92860286848B3E868406829890844B5
:109030003B490968401A002809DDE86880883849FA
:109040000988081A288129896868FDF7ABFBA18D7A
:10905000A06A014434480088314A126810448142B1
:109060003DD22968C9688889FCF7A9FB00F0010096
:10907000B0B12968C968888901E031E02FE0FCF7C8
:109080009EFB00F03E0B5846FCF779FB2968C96847
:1090900089894CF2FF02114008432968C968888118
:1090A000208DA18D08441E490988401A296808812D
:1090B0002A6811895068FDF775FB2968C968888995
:1090C000FCF77DFB00F0030008B1012000E0002068
:1090D0002968098908441449088000BF00BF04E0DA
:1090E0002F462D68002D7FF425AF17E0204600F0B5
:1090F00068F913E00A49A06A0968081A08D4A18D22
:10910000A06A0844401E06490968081A002805DDBF
:1091100000BFA07F40F00200A07700BFBDE8FE8F37
:10912000D0000020DCF60020DA0000202DE9F0411C
:1091300007460D4614461E463CB12189284600F0DC
:109140000CF82046FDF766FA05E026B92846FDF73B
:109150002FFFBDE8F0810020FBE770B504460E4606
:1091600000BF00BF00BF00BFA08D3044A085A08D10
:1091700042F23821884201DD0846A085204600F0F1
:1091800099FB054640F68E00854208DB00BFA07FB4
:1091900040F00200A07700BF2046FEF771FD70BDD1
:1091A0002DE9F0410446206F08B9BDE8F081256F34
:1091B0002868206704F16C0600E03668306858B112
:1091C0003168C9684868FCF7F4FA0746E9684868F6
:1091D000FCF7EFFA381AF0D4306828603560286858
:1091E00010B90020A4F86A0094F84600401C84F8E6
:1091F00046000020A06300BFD7E710B50446206FEB
:1092000090B3A07F00F0040070BB2046FFF7C8FFBA
:10921000B4F84C00B4F86010884207DDB4F8600080
:1092200000EBD0714910A4F84E1006E0B4F84C00E1
:1092300000EBD0714910A4F84E10B4F84E00E18E46
:109240004900884204DAE08E4004000CA4F84E0085
:10925000B4F84E00E18E032202FB0100A4F84C009A
:10926000A07F40F00400A07710BD70B50446206FC9
:1092700000B970BD256F00E02D6828680028FBD17B
:10928000E06E2860206FE0660020206794F84600BA
:10929000401C84F846000020A0632046FEF7F0FC46
:1092A00000BFE6E72DE9FC5F81460E46174698466B
:1092B000DDE90CAB002214210120FCF7EBFF054691
:1092C0000DB9BDE8FC9F00BF00BF6C685046FCF7BD
:1092D00056FA20805846FCF752FA60804846FCF760
:1092E00041FA60603046FCF73DFAA06045F2140098
:1092F000FCF745FAA08143F62200E081002020829D
:1093000060820B48B0F87800401C0949A1F8780049
:1093100006200021FF234246CDE9001039462846A9
:10932000FCF772F82846FDF775F900BFC9E70000A1
:10933000B8F5002070B5054640F29D4208A1042012
:10934000FCF754FD04460CB9002070BD95E80F00F1
:1093500084E80F006068FDF761FA2046F5E7000039
:109360002E2E5C2E2E5C5372635C5573725C4472BD
:10937000697665725C55704472697665725C6C776B
:1093800069705C636F72655C7463702E63000000CB
:1093900010B5044644B1606810B16068FDF73AF951
:1093A00021460420FCF79CFC10BD70B5044605E086
:1093B00025682046FFF7ECFF2C4600BF002CF7D1B4
:1093C00070BD2DE9FC4104460027206DFCF7CAF969
:1093D00080464346002239462046FEF731FD0546C9
:1093E00015B9B81EBDE8FC816E68A07F20F00300AF
:1093F000A0770621607ACDE90001A37A221D2146DB
:109400002846FCF701F82846FDF704F90020E9E7B3
:1094100070B50446E06ED8B1E56E00E02D682868AE
:109420000028FBD1E9688889FCF7C9F900F007003A
:1094300068B90120FCF7A3F9E96889890843E9685C
:109440008881A07F40F02000A077002070BD00BF81
:1094500001212046FDF732FFF8E700002DE9FE4F1D
:1094600000200290CA480068401CC9490860C948E9
:109470000078401CC749087000BF0025C648046832
:1094800058E100BF00BF00BF00BF00BF00BF94F89D
:109490002100C0490978884201D1E4684AE1BD4809
:1094A000007884F821000026B146207E022806D1EB
:1094B00094F84600062802D1701CC6B26BE094F8FE
:1094C00046000C2802D1701CC6B264E094F89D00DE
:1094D00000281BDD14F89C0F401C20702178607858
:1094E0009C3C401EAD4A105C814254DB002084F855
:1094F0009C0094F89D00072804D294F89D00401C1D
:1095000084F89D00204600F0FDF944E0B4F93400F1
:10951000002803DBA08E401C00B2A086206FD0B3D1
:10952000B4F93400B4F94410884234DB207E0228B8
:109530000CD040346088B4F9001000EBE100A17950
:10954000974A515C884000B2A080403C0020A08631
:10955000B4F84C00B4F86010884202DAB4F84C0059
:1095600001E0B4F8600082464FEA6A00A4F84E00B9
:10957000B4F84E00E18EB0EB410F06DAE08E4FF604
:10958000FF7101EA4000A4F84E00E08EA4F84C0000
:109590002046FFF76AFE207E06280BD1A07F00F050
:1095A000100038B17A49606A0968081A282801D978
:1095B000701CC6B2207A00F00800A8B3207E0428F0
:1095C00002D0207E07282FD12434D4E91C21E06E5C
:1095D00001FB02004FF4FA71B0FBF1F054F82419CA
:1095E0006B4A1268511A884206D2701CC6B209F141
:1095F000010000F0FF0917E094F89E10D4E924025E
:1096000001FB02004FF4FA71B0FBF1F0604A616AAD
:109610001268511A884207D22046FEF7C5F994F81D
:109620009E00401C84F89E00606F78B15849606AC3
:109630000968081AB4F9441001EB4101B0EB410F7D
:1096400004D3606FFFF7B1FE00206067207E03281F
:1096500007D14F49606A0968081A282801D9701C87
:10966000C6B2207E092807D14949606A0968081AEC
:10967000F02801D9701CC6B2A6B32046FEF7E8FC5C
:1096800025B100BF00BFE068E86004E000BF00BF94
:109690004149E0680860B9F1000F09D0A08B618BE7
:1096A000CDE90010231D2246A16A206DFFF7FAFDC7
:1096B000D4F88C80D4F810B02746E46839460220EC
:1096C000FCF70EFB00203749087000BFB8F1000F0F
:1096D00003D06FF009015846C04700BF31480078F9
:1096E00008B1CAE600E024E02546E468E87F401CB3
:1096F000E877E87F95F8201088421ADB0020E877A9
:109700002849087000BFD5F8880030B12946D5F83F
:10971000882028699047029001E00020029000BF55
:109720002048007800B1A8E6029810B92846FEF754
:10973000A7FA00BF002C7FF4A4AE00251A480468E5
:1097400022E000BF00BF00261149606A0968081ABC
:10975000F02801D9701CC6B2A6B12046FEF778FCED
:1097600025B100BF00BFE068E86004E000BF00BFB3
:109770000D49E06808602746E46839460220FCF796
:10978000AFFA01E02546E468002CDAD1BDE8FE8F8F
:10979000A8000020C2000020B400002075AB00002B
:1097A00068AB0000C0000020B800002010B50948D8
:1097B000006868B90848006810B90848006838B1FE
:1097C00001200449086000220549FA20FDF70CFA3F
:1097D00010BD0000EC000020B4000020B800002004
:1097E000399B00001CB504462148007800F00400B5
:1097F00008B100201CBD1E48007800F0020008B32C
:109800001C49A06A0968081A24D4A18DA06A0844DA
:1098100018490968081A00281CDC174800680088E5
:10982000154909684988CDE9001012480068134AB3
:1098300012888118124B134A13480068FFF732FD53
:109840000020D7E70A48007800F0010010B10F4867
:109850000068606209480088002807DDA07F40F0AA
:109860000200A0772046FEF70BFAC3E70020C1E70D
:10987000D8000020D0000020C8000020DA0000201E
:109880000001002004010020D4000020A8000020D6
:1098900010B5FDF7BDFD06480078401CC0B2044974
:1098A000087000F0010008B1FFF7D8FD10BD0000FE
:1098B000C100002010B501468B8D886AC218C88E81
:1098C00041F21C140B6BA04201DD204600E0C88E63
:1098D0001844101A04D4888DC885086B101A10BD5E
:1098E0000B6B886AC01A002802DD0020C88506E0DC
:1098F0008C6A0B6B181B00BF00BFC88500BF00201F
:10990000EDE700002DE9FC4705462C6F04B9EC6E2D
:109910000CB9BDE8FC87E1688889FBF750FF00F0CF
:10992000010018B1208908B9012000E0002080461C
:10993000B8F1000F01D1012000E000208146E0686D
:1099400043684A4600212846FEF77AFA064606B9D9
:10995000DFE77768B8F1000F09D01120FBF70FFFA0
:10996000B9894CF2FF0211400843B8810DE07068DC
:1099700000F1140A616809892289891A8BB20122CF
:1099800051466068FCF7FDFD00BF0B48B0F8780059
:10999000401C0949A1F8780006200021CDE90010FB
:1099A000AB7A2A1D29463046FBF72EFD3046FCF7E0
:1099B00031FE00BFADE70000B8F500202DE9F04111
:1099C00005460E4617461548FDF798F8002822D0A0
:1099D000E12213A10720FCF709FA04461CB94FF055
:1099E000FF30BDE8F08105202070A560E66027B15A
:1099F00021460A48FDF75EF80BE021460748FDF7CF
:109A000069F830B121460720FCF76AF94FF0FF30C2
:109A1000E7E70020E5E76FF00500E2E77C000020C3
:109A20002E2E5C2E2E5C5372635C5573725C4472F6
:109A3000697665725C55704472697665725C6C77A4
:109A400069705C6170695C74637069702E6300009A
:109A500038B504460D46FBF798FE0E4804600E48E4
:109A60000560C8210D48FCF7FFFF08B100BF00BF2B
:109A700001210B48FDF75EF808B100BF00BF0520CB
:109A80004FF4006300220749009007A0FDF772F829
:109A900038BD000074000020780000207C00002009
:109AA00080000020719B000074637069705F7468AF
:109AB000726561640000000070B505460E461148ED
:109AC000FDF71CF810B96FF0050070BDC0220EA1A3
:109AD0000820FCF78BF9044614B94FF0FF30F4E787
:109AE00001202070A560E66021460648FCF7F2FFE1
:109AF00030B121460820FCF7F3F84FF0FF30E4E7DF
:109B00000020E2E77C0000202E2E5C2E2E5C53729B
:109B1000635C5573725C4472697665725C5570441F
:109B200072697665725C6C7769705C6170695C748F
:109B3000637069702E63000010B50446FFF7A8FE3D
:109B40000748006810B90748006828B10022064994
:109B5000FA20FDF749F802E000200449086010BD32
:109B6000B4000020B8000020399B0000EC00002069
:109B700008B53A48006820B1394800683749096893
:109B800088474FF4FA70F9F7FBF900213548FCF7E4
:109B900025FF61E03348FCF7E7FF69463248FDF7EF
:109BA00099F800212F48FCF719FF00980078072842
:109BB0004ED2DFE800F0040C232B353F4800009A1A
:109BC0009268101D009A92681168884743E00098D7
:109BD000C06890F8350000F0600028B1009AD2E922
:109BE0000201FBF701F904E0009AD2E90201FBF758
:109BF00007FB08200099FCF773F82CE0009A9268A4
:109C0000101D009A92681168884724E0009B083371
:109C100007CBFCF7E9FF07200099FCF761F81AE091
:109C2000009AD2E90301FDF7A3F807200099FCF799
:109C300057F810E0009AD2E90210884707200099EF
:109C4000FCF74EF807E0009AD2E90210884702E0DC
:109C500000BF00BF00BF00BF9CE7000074000020F1
:109C600078000020800000207C00002070B50546B0
:109C70002C4600BF6068B0F1005F03D30F496068F5
:109C8000884215D3298903221046FCF703FB0446BA
:109C90004CB129462046FCF714FC06461EB120466E
:109CA000FCF7B8FC00242846FCF7B4FC204670BD45
:109CB0002468002CDED12846F9E7000000000720C8
:109CC00070B504463748FAF75BF83748F7F774FF82
:109CD0003648F7F771FF60213548F7F795FF062002
:109CE00084F82E0004F12F0200213248F7F7C8FC57
:109CF00040F2DC50A085322084F83500F8F728F8CF
:109D0000122200212B48F7F70FFE054613220021EF
:109D10002848F7F709FE0546112200212548F7F7E4
:109D200003FE054645F003052B461122002121487C
:109D3000F7F713FE3C23122200211E48F7F70DFE11
:109D4000122200211B48F7F7EFFD05464FF4826110
:109D50001848F7F7FFFC00211648F7F795FD06466F
:109D600031461448F7F752FD1248F7F73AFE11480A
:109D7000F7F721FE10490F48F7F765FD3820F8F78F
:109D80008DF8F8F7C5F80D492820F6F787FE28204A
:109D9000F6F71AFC4FF49053002211460548F7F7E6
:109DA000DCFD70BD090800F0051809000514090064
:109DB0000010064000C00E40C30100808155000025
:109DC00010B5044600BF00BF0A48A062742084F8A2
:109DD0003600692137200155074860610748A061B6
:109DE00004F12F00034908602046FFF769FF0020B7
:109DF00010BD00003801002031480000C1A1000062
:109E000070B505460C46AE6A04F4803020B11048A7
:109E10000068401C0E49086004F4004020B10D4861
:109E20000068401C0B49086004F0004010B128464F
:109E300000F012F804F0010010B1304600F068F8AC
:109E400004F4E07010B1284600F0A6F870BD0000E0
:109E50004401002048010020FEB5054612220021E1
:109E60002748F7F761FD0646102200212448F7F73E
:109E70005BFD0446012200212148F7F755FD074606
:109E800000BF06F4005098B104F0010040B1012079
:109E90001C490870012229461B48FFF78FFD07E087
:109EA000002018490870012229461848FFF786FD4E
:109EB00006F4A05018B36B4601AA02A91048F7F7A0
:109EC0000FFC04F0020020B1029820F480400290C0
:109ED00003E0029840F48040029004F0040020B1B6
:109EE000029840F40060029003E0029820F40060C1
:109EF00002900348DDE900320299F7F711FCFEBD3C
:109F000000C00E404C010020FF610000D561000040
:109F100070B505466C68002639E0A16801EBC10107
:109F2000206850F8210000F0004000B132E0A16844
:109F300001EBC101206800EB8100006AE0B1A1687B
:109F400001EBC101206800EB810090F8200000F0D7
:109F5000010040B9A26802EBC202216801EB820154
:109F6000086AFCF757FB0020A26802EBC2022168D6
:109F700001EB8201086200E00CE0A068401CA060D8
:109F8000D4E90110884201D10020A060761C6068ED
:109F9000B042C2D800BF70BD2DE9F0410546AE6A9F
:109FA000B468A06810B1A068401E01E06068401E5F
:109FB0000746FAE0A16801EBC101206800EB8100CF
:109FC000006A002870D0A16801EBC101206850F838
:109FD000210000F0004000B1EBE0A16801EBC101FD
:109FE000206850F8210000F48070F8B1A16801EBFE
:109FF000C101206850F82100C0F30D40A26802EBB7
:10A00000C202216801EB8201096A4881A16801EB63
:10A01000C101206800EB8100006A4089A26802EB60
:10A02000C202216801EB8201096A08816248006866
:10A0300098B1A26802EBC202206800EB8200016ABC
:10A040005D480068FCF718FA5B480068A26802EBFC
:10A05000C202216801EB82010862A16801EBC10123
:10A06000206800EB8100006A53490860A16801EB99
:10A07000C101206850F8210000F48070A0B1A168EF
:10A0800001EBC101206850F8210000F4004060B1EC
:10A0900049480068FCF7BEFA4848C088401C474958
:10A0A000C8800020444908601AE044484088401CA9
:10A0B00042494880294640480068FFF7FDFC60B1EE
:10A0C0003D480068FCF7A6FA3C488089401C3B49A3
:10A0D00088810846C088401CC88000203649086036
:10A0E000032240F2EC511046FCF7D4F8A26802EBD0
:10A0F000C202216801EB820108624FF48040A2682D
:10A1000002EBC202216801EB82014860A16801EB09
:10A11000C101206800EB8100006A70B3A16801EB07
:10A12000C101206800EB8100006A4068A26802EB70
:10A13000C202216801EB82018860A16801EBC101C4
:10A14000206800EB81004068A26802EBC20221682F
:10A1500001EB8201096A49890843A26802EBC20245
:10A16000216801EB820148604FF00040A26802EBD9
:10A17000C202216841F822000EE0FFE70020A26839
:10A1800002EBC202216801EB820188600B488089E2
:10A19000401C0A4988810CE0A068401CA060D4E9FA
:10A1A0000110884201D10020A060A068B8427FF46D
:10A1B00001AF00BFBDE8F08150010020B8F50020DC
:10A1C0002DE9F84F81460E4600200090FCF702FC76
:10A1D00000903046FCF722FB3046FFF747FD06466D
:10A1E0005EB94E488089401C4C4988810098FCF734
:10A1F00027FC4FF0FF30BDE8F88FD9F828406068A1
:10A2000000686168C96801EBC10100EB8105286A3B
:10A2100068B13046FCF7FEF940488089401C3F4950
:10A2200088810098FCF70CFC4FF0FF30E3E73046E4
:10A23000FCF73EF90746606880686168C968884233
:10A2400005D9606880686168C968401A06E060687E
:10A25000C068C0F118006168896808448346BB453E
:10A260000DD23046FCF7D6F92C488089401C2B498A
:10A2700088810098FCF7E4FB4FF0FF30BBE74FF01C
:10A28000010A4FF080502860B04638E060680068EE
:10A290006168C96801EBC10100EB8105B8F80A00EB
:10A2A0006860D8F80400A860BAF1000F05D04FF03C
:10A2B000000A4FF08050286001E0002028602868E4
:10A2C00040F4500028607F1ED8F800806068C068A5
:10A2D000401C6168C8606068C068182802D100200E
:10A2E0006168C8602FB9286840F0C04028602E62BD
:10A2F00001E0701C2862286840F000402860002FB0
:10A30000C4D10748F7F769FB04480088401C03499B
:10A3100008800098FCF794FB00206CE7B8F500205B
:10A3200000C00E40704700002DE9FF5F05460E4655
:10A330007B48B0F86200401C81B27948A0F86210F6
:10A34000D5F804B029899BF8000000F00F0008221E
:10A3500002EB8000814208DB9BF800000007800EC2
:10A3600041422846FCF7BBF990B16D48B0F86A004D
:10A37000401C81B26A48A0F86A10B0F86600401C20
:10A3800081B26748A0F866102846FCF743F9C4E09C
:10A39000D5F80490634908683146FAF70AFF804609
:10A3A000B9F80000FBF70BFA0390B9F80200FBF7CD
:10A3B00006FA029000270020019082465A4804685D
:10A3C0004CE000200190618A0298814223D1B8F1CB
:10A3D000000F02D1ACB1206898B1524920680968D9
:10A3E00088420ED0B8F1000F15D054B1206840B1AA
:10A3F0002168B06801404B480068B2681040814253
:10A4000009D101200190BAF1000F04D1207C00F0A5
:10A41000040000B9A2460198F0B1A18A03988142D4
:10A420001AD1201D30B1606820B1404960680968C8
:10A43000884211D13FB1E068F8603B480068E060B5
:10A440003948046007E03648B0F87600401C81B215
:10A450003348A0F8761003E02746E468002CB0D11A
:10A4600000BF04B9544624B92E497068096888426F
:10A470004FD16FF007012846FCF731F968B100BFF2
:10A4800000BF2748B0F86600401C81B22448A0F8FD
:10A4900066102846FCF7BEF83FE074B1A06940B1F1
:10A4A00003980090214B2A462146D4E906C0E04794
:10A4B00032E02846FCF7AEF82FE0B8F1000F15D1D6
:10A4C0001848007800F0F000E0280FD09BF800005A
:10A4D00000F00F00082202EB80012846FCF7FFF88D
:10A4E00000BF00BF03212846FAF7F2FC0C48B0F881
:10A4F0007000401C81B20A48A0F87010B0F86600E5
:10A50000401C81B20648A0F866102846FCF782F885
:10A5100002E02846FCF77EF800BFBDE8FF9F000080
:10A52000B8F5002004010020F40000200001002004
:10A5300010B505490120F6F7FDFF4FF4E131012088
:10A54000F7F792F810BD0000801A06000090D003C3
:10A550000C00000000EA32060000000080D1F00884
:10A560000400000000400040100000000080054092
:10A570001000000000500040110000000090054055
:10A5800011000000006000401200000000A0054023
:10A5900012000000007000401300000000B00540F1
:10A5A00013000000004002401400000000C00540FD
:10A5B00014000000005002402E00000000D00540B2
:10A5C0002E000000006002402F00000000E0054067
:10A5D0002F000000007002403000000000F0054035
:10A5E0003000000000D0034046000000000006409C
:10A5F0004600000000100640470000000020064012
:10A6000048000000003006407F0000000040064087
:10A6100080000000005006408400000000600640FA
:10A620008C00000000400040100000000080054049
:10A630001000000000500040110000000090054094
:10A6400011000000006000401200000000A0054062
:10A6500012000000007000401300000000B0054030
:10A6600013000000004002401400000000C005403C
:10A6700014000000005002402E00000000D00540F1
:10A680002E000000006002402F00000000E00540A6
:10A690002F000000007002403000000000F0054074
:10A6A0003000000000D003404300000000000640DE
:10A6B0004300000000100640440000000020064057
:10A6C00045000000003006405800000000400640F1
:10A6D00059000000005006405C0000000060064089
:10A6E00064000000007006406C000000008006401E
:10A6F0006D000000009006407F0000000040004018
:10A70000008005400050004000900540006000407F
:10A7100000A005400070004000B00540004002402D
:10A7200000C005400050024000D0054000600240DB
:10A7300000E005400070024000F0054000D00340FA
:10A7400000000640001006400010064000200640B1
:10A750000020064000300640003006400040064021
:10A760000040064000500640005006400060064091
:10A770000060064000700640007006400080064001
:10A780000080064000900640009006400007000050
:10A7900000060000000500000004000000030000A7
:10A7A00000020000000100000000000000000000A6
:10A7B00018ED00E01CED00E020ED00E000E400E01A
:10A7C00004E400E008E400E00CE400E010E400E051
:10A7D00014E400E018E400E01CE400E020E400E001
:10A7E00024E400E028E400E02CE400E030E400E0B1
:10A7F00034E400E038E400E03CE400E040E400E061
:10A8000044E400E048E400E04CE400E050E400E010
:10A8100054E400E058E400E05CE400E060E400E0C0
:10A8200064E400E068E400E06CE400E070E400E070
:10A8300074E400E078E400E07CE400E080E400E020
:10A8400084E400E088E400E000E100E004E100E0EE
:10A8500008E100E00CE100E010E100E080E100E050
:10A8600084E100E088E100E08CE100E090E100E0BC
:10A8700000E200E004E200E008E200E00CE200E0B8
:10A8800010E200E080E200E084E200E088E200E024
:10A890008CE200E090E200E0000001000200010014
:10A8A0000300010002000100040001000200010099
:10A8B0000300010002000100050001000200010088
:10A8C0000300010002000100040001000200010079
:10A8D0000300010002000100060001000200010067
:10A8E0000300010002000100040001000200010059
:10A8F0000300010002000100050001000200010048
:10A900000300010002000100040001000200010038
:10A910000300010002000100070001000200010025
:10A920000300010002000100040001000200010018
:10A930000300010002000100050001000200010007
:10A9400003000100020001000400010002000100F8
:10A9500003000100020001000600010002000100E6
:10A9600003000100020001000400010002000100D8
:10A9700003000100020001000500010002000100C7
:10A9800003000100020001000400010002000100B8
:10A99000030001000200010001000000785634129B
:10A9A0000100400001001800000601000100100035
:10A9B000140002000A0001003F0001000100050030
:10A9C00001001800780001000400010004001800D4
:10A9D00008000100040001000100010080000100E6
:10A9E000160001000100800001000100010040008C
:10A9F0005800E80301001A7201001000010008006D
:10AA0000E803280080020800400022191C002000F2
:10AA1000A0001C00100010003000140014001000F2
:10AA200030001C06040004000600040014000A00A4
:10AA30000800080010001000300014006465746500
:10AA400063746564206D656D70206F766572666CE9
:10AA50006F7720696E20706F6F6C2000000000001F
:10AA600000000000000000000000000000000000E6
:10AA700000000000000000000000000000000000D6
:10AA800000000000000000000000000000000000C6
:10AA900000000000000000000000000000000000B6
:10AAA00000000000000000000000000000000000A6
:10AAB00000000000000000000000000064657465F4
:10AAC00063746564206D656D7020756E6465726673
:10AAD0006C6F7720696E20706F6F6C200000000033
:10AAE0000000000000000000000000000000000066
:10AAF0000000000000000000000000000000000056
:10AB00000000000000000000000000000000000045
:10AB10000000000000000000000000000000000035
:10AB20000000000000000000000000000000000025
:10AB3000000000000000000000000000BCAB0000AE
:10AB4000E4AB000004AC0000C4AB0000B0AB0000FC
:10AB500098AB0000A4AB0000F8AB0000D0AB000045
:10AB6000D8AB0000ECAB00000102030405060707A8
:10AB7000070707070703060C18306078B0000020AD
:10AB8000AC000020B4000020B8000020FFFFFFFF51
:10AB9000FFFF00000000000046494E5F5741495446
:10ABA0005F31000046494E5F574149545F32000013
:10ABB00045535441424C495348454400434C4F533C
:10ABC0004544000053594E5F524356440000000074
:10ABD000434C4F53494E47004C4153545F41434B04
:10ABE000000000004C495354454E000054494D4567
:10ABF0005F57414954000000434C4F53455F574154
:10AC00004954000053594E5F53454E540000000014
:10AC100030AC000000000020D00100007C040000E7
:10AC200064AC0000D0010020603701004841000002
:10AC300001A5021EC00B486E194C1AFF011310012A
:10AC4000B720701E012018F6D0210120081A1828FC
:10AC50001A2804016C1DC0A80164A329084201E35D
:04AC60007A04000072
:0400000500000201F4
:00000001FF
